:020000040000FA
:0408000070EF0BF09A
:1008100003B273EF05F0F2B491EF05F09EB099EFDB
:1008200005F09EB2A1EF05F0F2A81AEF04F0F2B2C3
:1008300021EF04F0F2B01FEF04F01FEF0BF0F2967F
:10084000F290CD90F2929EA02BEF04F00101533F65
:100850002BEF04F0542BB2C1B6F1B3C1B7F1B4C160
:10086000B8F1B5C1B9F1AEC1B2F1AFC1B3F1B0C128
:10087000B4F1B1C1B5F1AAC1AEF1ABC1AFF1ACC138
:10088000B0F1ADC1B1F1A6C1AAF1A7C1ABF1A8C148
:10089000ACF1A9C1ADF1A2C1A6F1A3C1A7F1A4C158
:1008A000A8F1A5C1A9F19EC1A2F19FC1A3F1A0C168
:1008B000A4F1A1C1A5F19AC19EF19BC19FF19CC178
:1008C000A0F19DC1A1F1CECF9AF1CFCF9BF153C141
:1008D0009CF154C19DF1CF6ACE6A0101536B546BF8
:1008E0009E90CD800FBC0F8E0FBA7AEF04F00F8A66
:1008F0001FEF0BF013880F8C0FBEB7EF04F09AC1F7
:100900009EF19BC19FF19CC1A0F19DC1A1F19EC12F
:10091000A2F19FC1A3F1A0C1A4F1A1C1A5F1A2C1FF
:10092000A6F1A3C1A7F1A4C1A8F1A5C1A9F1A6C1CF
:10093000AAF1A7C1ABF1A8C1ACF1A9C1ADF1AAC19F
:10094000AEF1ABC1AFF1ACC1B0F1ADC1B1F1AEC16F
:10095000B2F1AFC1B3F1B0C1B4F1B1C1B5F1B2C13F
:10096000B6F1B3C1B7F1B4C1B8F1B5C1B9F1010184
:100970005E6B5F6B606B616B9A515E279B515F236F
:100980009C5160239D5161239E515E279F515F239F
:10099000A0516023A1516123A2515E27A3515F237F
:1009A000A4516023A5516123A6515E27A7515F235F
:1009B000A8516023A9516123AA515E27AB515F233F
:1009C000AC516023AD516123AE515E27AF515F231F
:1009D000B0516023B1516123B2515E27B3515F23FF
:1009E000B4516023B5516123B6515E27B7515F23DF
:1009F000B8516023B9516123D8900101613360334C
:100A00005F335E33D8900101613360335F335E330F
:100A1000D8900101613360335F335E3300C10CF164
:100A200001C10DF102C10EF103C10FF104C110F1BA
:100A300005C111F106C112F107C113F108C114F18A
:100A400009C115F10AC116F10BC117F134C135F115
:100A500011B836EF05F00101620E046F010E056F4B
:100A6000000E066F000E076F3FEF05F00101A70EA5
:100A7000046F020E056F000E066F000E076F5EC159
:100A800000F15FC101F160C102F161C103F172ECDB
:100A90002DF003BF04D01CBE02D01CA0108C11A0EE
:100AA00057EF05F010BA57EF05F00F80108A0CC110
:100AB00000F10DC101F10EC102F10FC103F110C12E
:100AC00004F111C105F112C106F113C107F114C1FE
:100AD00008F115C109F116C10AF117C10BF135C1B1
:100AE00034F11FEF0BF00392ABB2AB98AB8803016C
:100AF00003EE00F080517F0BE92604C0EFFF802B4E
:100B00008151805D700BD8A48B8200008051815D83
:100B1000700BD8A48B9281518019D8B407901FEF25
:100B20000BF0F2940101453F1FEF0BF0462B1FEF36
:100B30000BF09E900101533F1FEF0BF0542B1FEF62
:100B40000BF09E9211B835EF08F0040066A1A9EFF2
:100B500005F08BB4B3EF05F010ACB3EF05F08B8468
:100B6000109CB4EF05F08B94077C07ACCFEF05F039
:100B7000C274C2B4C9EF05F0C3CFB7F5C4CFB8F59E
:100B80000501D890B833B733D890B833B733D0EF26
:100B900005F0C3CF55F1C4CF56F1D0EF05F0C282B6
:100BA00007B442EF06F047C14BF148C14CF149C1CF
:100BB0004DF14AC14EF15EC162F15FC163F160C1A6
:100BC00064F161C165F113A8E8EF05F0138C139887
:100BD0009AC1BAF19BC1BBF19CC1BCF19DC1BDF1F1
:100BE0009EC1BEF19FC1BFF1A0C1C0F1A1C1C1F1C1
:100BF000A2C1C2F1A3C1C3F1A4C1C4F1A5C1C5F191
:100C0000A6C1C6F1A7C1C7F1A8C1C8F1A9C1C9F160
:100C1000AAC1CAF1ABC1CBF1ACC1CCF1ADC1CDF130
:100C2000AEC1CEF1AFC1CFF1B0C1D0F1B1C1D1F100
:100C3000B2C1D2F1B3C1D3F1B4C1D4F1B5C1D5F1D0
:100C4000B6C1D6F1B7C1D7F1B8C1D8F1B9C1D9F1A0
:100C5000B7C5B9F5B8C5BAF5B9C5BBF5BAC5BCF5E0
:100C6000010155515B2756515C23E86A5D230E2E26
:100C700042EF06F05CC157F15DC158F15B6B5C6BF4
:100C80005D6B078E0201002F1FEF0BF03C0E006F13
:100C90001D50E00BE00AE86612881BBE02D01BB4B0
:100CA000108E00C10CF101C10DF102C10EF103C1A2
:100CB0000FF104C110F105C111F106C112F107C114
:100CC00013F108C114F109C115F10AC116F10BC1E4
:100CD00017F134C135F181AA2CEF07F037A0FCEFF2
:100CE00006F005012F51000AD8B42CEF07F00501DA
:100CF0002F51010AD8B4ACEF06F005012F51020ABA
:100D0000D8B4EEEF06F005012F51030AD8B4EEEF88
:100D100006F005012F51040AD8B4EEEF06F00501E4
:100D20002F51050AD8B4EEEF06F005012F51060A3F
:100D3000D8B4EEEF06F005012F51070AD8B4EEEF54
:100D400006F005012F51320AD8B4AAEF06F02F6B36
:100D50002CEF07F02CEF07F005015767B7EF06F00F
:100D60005867B7EF06F05967B7EF06F05A67BBEF61
:100D700006F02CEF07F05BC500F15CC501F15DC525
:100D800002F15EC503F10101010E046F000E056F53
:100D9000000E066F000E076F72EC2DF000C15BF5C0
:100DA00001C15CF502C15DF503C15EF5010100679B
:100DB000E1EF06F00167E1EF06F00267E1EF06F010
:100DC00003672CEF07F057C55BF558C55CF559C5AF
:100DD0005DF55AC55EF515802CEF07F00001165041
:100DE000000AD8B4FCEF06F000011650030AD8B48C
:100DF000FCEF06F02CEF07F00FBE11EF07F010A08C
:100E000016EF07F0010147670DEF07F048670DEF98
:100E100007F049670DEF07F04A6711EF07F016EF8B
:100E200007F007AE16EF07F029EF07F00501312FA5
:100E30002CEF07F03C0E316F302F2CEF07F0010143
:100E4000000E626FE00E636FA50E646F010E656F9A
:100E500013880501306B162A0501666B37B732EF30
:100E600007F066810CC100F10DC101F10EC102F164
:100E70000FC103F110C104F111C105F112C106F156
:100E800013C107F114C108F115C109F116C10AF126
:100E900017C10BF135C134F100C10CF101C10DF1E5
:100EA00002C10EF103C10FF104C110F105C111F12E
:100EB00006C112F107C113F108C114F109C115F1FE
:100EC0000AC116F10BC117F134C135F101018E676A
:100ED00071EF07F08F6771EF07F0906771EF07F020
:100EE000916775EF07F0A6EF07F092C100F193C18B
:100EF00001F194C102F195C103F10101010E046FEA
:100F0000000E056F000E066F000E076F72EC2DF0DD
:100F100000C192F101C193F102C194F103C195F1B5
:100F2000010100679BEF07F001679BEF07F0026785
:100F30009BEF07F00367A6EF07F08EC192F18FC118
:100F400093F190C194F191C195F10F80D57ED5BEFA
:100F50006ED0D6CF47F1D7CF48F145C149F1E86A05
:100F6000E8CF4AF1138A1CBE02D01CA0108C10904E
:100F700047C100F148C101F149C102F14AC103F181
:100F800001010A0E046F000E056F000E066F000EC1
:100F9000076F72EC2DF003AF1080010154A7DDEF55
:100FA00007F00F9A0F9C0F9E0101000E5E6F600EFE
:100FB0005F6F3D0E606F080E616F010147BFEDEF7F
:100FC00007F04867EDEF07F04967EDEF07F04A6774
:100FD000EDEF07F0F28812EF08F0F2985E6B5F6BAE
:100FE000606B616B9A6B9B6B9C6B9D6B9E6B9F6B3D
:100FF000A06BA16BA26BA36BA46BA56BA66BA76B7D
:10100000A86BA96BAA6BAB6BAC6BAD6BAE6BAF6B2C
:10101000B06BB16BB26BB36BB46BB56BB66BB76BDC
:10102000B86BB96BD76AD66A0101456B466B0CC1C8
:1010300000F10DC101F10EC102F10FC103F110C1A8
:1010400004F111C105F112C106F113C107F114C178
:1010500008F115C109F116C10AF117C10BF135C12B
:1010600034F11FEF0BF01FEF0BF00201002F83EFA5
:101070000AF0D59ED6CF47F1D7CF48F145C149F107
:10108000E86AE8CF4AF1138AD76AD66A0101456B4C
:10109000466BD58E1D50E00BE00AE86612881BBE39
:1010A00002D01BB4108E1AAE1F8C00C10CF101C10E
:1010B0000DF102C10EF103C10FF104C110F105C120
:1010C00011F106C112F107C113F108C114F109C1F0
:1010D00015F10AC116F10BC117F134C135F10FA09A
:1010E000109A11B87FEF08F00101620E046F010E33
:1010F000056F000E066F000E076F88EF08F0010104
:10110000A70E046F020E056F000E066F000E076F2C
:1011100047C100F148C101F149C102F14AC103F1DF
:1011200072EC2DF003BF9BEF08F01CBE02D01CA098
:10113000108C11B00F800CC100F10DC101F10EC176
:1011400002F10FC103F110C104F111C105F112C187
:1011500006F113C107F114C108F115C109F116C157
:101160000AF117C10BF135C134F102013C0E006FD9
:1011700000C10CF101C10DF102C10EF103C10FF16B
:1011800004C110F105C111F106C112F107C113F13B
:1011900008C114F109C115F10AC116F10BC117F10B
:1011A00034C135F181AA8BEF09F037A05BEF09F06C
:1011B00005012F51000AD8B48BEF09F005012F511A
:1011C000010AD8B413EF09F005012F51020AD8B46F
:1011D00055EF09F005012F51030AD8B455EF09F076
:1011E00005012F51040AD8B455EF09F005012F511C
:1011F000050AD8B455EF09F005012F51060AD8B4F5
:1012000055EF09F005012F51070AD8B455EF09F041
:1012100005012F51320AD8B411EF09F02F6B8BEF73
:1012200009F08BEF09F0050157671EEF09F05867C9
:101230001EEF09F059671EEF09F05A6722EF09F017
:101240008BEF09F05BC500F15CC501F15DC502F1F2
:101250005EC503F10101010E046F000E056F000E63
:10126000066F000E076F72EC2DF000C15BF501C137
:101270005CF502C15DF503C15EF50101006748EF51
:1012800009F0016748EF09F0026748EF09F00367CA
:101290008BEF09F057C55BF558C55CF559C55DF591
:1012A0005AC55EF515808BEF09F0050130675BEFDD
:1012B00009F08BEF09F00FBE70EF09F010A075EF89
:1012C00009F0010147676CEF09F048676CEF09F01E
:1012D00049676CEF09F04A6770EF09F075EF09F0A4
:1012E00007AE75EF09F088EF09F00501312F8BEF9C
:1012F00009F03C0E316F302F8BEF09F00101000E29
:10130000626FE00E636FA50E646F010E656F138848
:101310000501306B15800501666B37B791EF09F059
:1013200066810CC100F10DC101F10EC102F10FC1C6
:1013300003F110C104F111C105F112C106F113C18D
:1013400007F114C108F115C109F116C10AF117C15D
:101350000BF135C134F100C10CF101C10DF102C135
:101360000EF103C10FF104C110F105C111F106C165
:1013700012F107C113F108C114F109C115F10AC135
:1013800016F10BC117F134C135F101018E67D0EFB1
:1013900009F08F67D0EF09F09067D0EF09F09167FF
:1013A000D4EF09F005EF0AF092C100F193C101F109
:1013B00094C102F195C103F10101010E046F000E09
:1013C000056F000E066F000E076F72EC2DF000C166
:1013D00092F101C193F102C194F103C195F10101B0
:1013E0000067FAEF09F00167FAEF09F00267FAEF18
:1013F00009F0036705EF0AF08EC192F18FC193F1F6
:1014000090C194F191C195F10F80109047C100F106
:1014100048C101F149C102F14AC103F101010A0EBB
:10142000046F000E056F000E066F000E076F72EC62
:101430002DF003AF1080010154A72BEF0AF00F9A93
:101440000F9C0F9E0101000E5E6F600E5F6F3D0EE0
:10145000606F080E616F47C100F148C101F149C1D9
:1014600002F14AC103F10101140E046F050E056F6C
:10147000000E066F000E076F72EC2DF003AF44EF05
:101480000AF0F28869EF0AF0F2985E6B5F6B606BAE
:10149000616B9A6B9B6B9C6B9D6B9E6B9F6BA06B48
:1014A000A16BA26BA36BA46BA56BA66BA76BA86BC0
:1014B000A96BAA6BAB6BAC6BAD6BAE6BAF6BB06B70
:1014C000B16BB26BB36BB46BB56BB66BB76BB86B20
:1014D000B96B0CC100F10DC101F10EC102F10FC1D8
:1014E00003F110C104F111C105F112C106F113C1DC
:1014F00007F114C108F115C109F116C10AF117C1AC
:101500000BF135C134F104008BB48EEF0AF010AC4E
:101510008EEF0AF08B84109C8FEF0AF08B94077C7F
:1015200007ACAAEF0AF0C274C2B4A4EF0AF0C3CFAA
:10153000B7F5C4CFB8F50501D890B833B733D89014
:10154000B833B733ABEF0AF0C3CF55F1C4CF56F180
:10155000ABEF0AF0C28207B41DEF0BF047C14BF1AD
:1015600048C14CF149C14DF14AC14EF15EC162F131
:101570005FC163F160C164F161C165F113A8C3EF9C
:101580000AF0138C13989AC1BAF19BC1BBF19CC1AC
:10159000BCF19DC1BDF19EC1BEF19FC1BFF1A0C113
:1015A000C0F1A1C1C1F1A2C1C2F1A3C1C3F1A4C1E3
:1015B000C4F1A5C1C5F1A6C1C6F1A7C1C7F1A8C1B3
:1015C000C8F1A9C1C9F1AAC1CAF1ABC1CBF1ACC183
:1015D000CCF1ADC1CDF1AEC1CEF1AFC1CFF1B0C153
:1015E000D0F1B1C1D1F1B2C1D2F1B3C1D3F1B4C123
:1015F000D4F1B5C1D5F1B6C1D6F1B7C1D7F1B8C1F3
:10160000D8F1B9C1D9F1B7C5B9F5B8C5BAF5B9C5F9
:10161000BBF5BAC5BCF5010155515B2756515C239A
:10162000E86A5D230E2E1DEF0BF05CC157F15DC122
:1016300058F15B6B5C6B5D6B078E1FEF0BF002C0AC
:10164000E0FF005001C0D8FF1000A6B225EF0BF05C
:101650000CC0A9FF0BC0A8FFA69EA69CA684F29E64
:10166000550EA76EAA0EA76EA682F28EA694A6B2FB
:1016700037EF0BF00C2A1200A96EA69EA69CA6803E
:10168000A8500C2A120004012C0E826FA8EC0EF058
:101690006DEC2EF00C503CEC0BF0E8CF00F10C5050
:1016A0003CEC0BF0E8CF01F101AF5CEF0BF0010176
:1016B000FF0E026FFF0E036F10EC2EF0296768EF2C
:1016C0000BF00401200E826FA8EC0EF06DEF0BF012
:1016D00004012D0E826FA8EC0EF01AEC2CF0120013
:1016E000376A076A0F6A106A116A126A136A156A02
:1016F000166A0F010D0EC16E860EC06E030EC26E0D
:101700000F01680E896E130E926E080E8A6EF30E2C
:10171000936E8B6A900E946EC80E3CEC0BF0E8CF83
:10172000E8FF1098E8A0108810A805D00E0E256ECE
:101730008E0E266E04D00F0E256E8F0E266EECECEC
:101740002EF0F18EF19EFC0E3CEC0BF0E8CF0BF08E
:101750000BA011800BA211820BA411840BA811887D
:10176000C90E3CEC0BF0E8CF1AF0CA0E3CEC0BF0C3
:10177000E8CF1BF0CB0E3CEC0BF0E8CF1CF0CC0E0E
:101780003CEC0BF0E8CF1DF0FB0E3CEC0BF0E8CF8F
:1017900038F0CE0E3CEC0BF0E8CF14F0CD0E3CEC64
:1017A0000BF0E8CF36F01F6A206A0E6A01015B6B0E
:1017B0005C6B5D6B576B586BF29A0101476B486B22
:1017C000496B4A6B4B6B4C6B4D6B4E6B4F6B506B5D
:1017D000516B526B456B466BD76AD66A0F01280E68
:1017E000D56EF28A9D90B00ECD6E01015E6B5F6B7F
:1017F000606B616B626B636B646B656B666B676B75
:10180000686B696B536B546BCF6ACE6A0F9A0F9CEF
:101810000F9E9D80760ECA6E9D8202013C0E006F67
:10182000CC6A160E3CEC0BF0E8CF00F1170E3CEC46
:101830000BF0E8CF01F1180E3CEC0BF0E8CF02F111
:10184000190E3CEC0BF0E8CF03F1010103AF43EFBD
:101850000CF06DEC2EF0160E0C6E00C10BF025ECAA
:101860000BF0170E0C6E01C10BF025EC0BF0180EEF
:101870000C6E02C10BF025EC0BF0190E0C6E03C1BF
:101880000BF025EC0BF000C18EF101C18FF102C10C
:1018900090F103C191F100C192F101C193F102C134
:1018A00094F103C195F11A0E3CEC0BF0E8CF00F176
:1018B0001B0E3CEC0BF0E8CF01F11C0E3CEC0BF0E6
:1018C000E8CF02F11D0E3CEC0BF0E8CF03F1010173
:1018D00003AF99EF0CF06DEC2EF01A0E0C6E00C1F8
:1018E0000BF025EC0BF01B0E0C6E01C10BF025EC80
:1018F0000BF01C0E0C6E02C10BF025EC0BF01D0E54
:101900000C6E03C10BF025EC0BF01A0E3CEC0BF047
:10191000E8CF00F11B0E3CEC0BF0E8CF01F11C0E00
:101920003CEC0BF0E8CF02F11D0E3CEC0BF0E8CFE5
:1019300003F100C196F101C197F102C198F103C111
:1019400099F1240EAC6E900EAB6E240EAC6E080EA8
:10195000B86E000EB06E1F0EAF6E0401806B816B0F
:101960000F01900EAB6E0F019D8A0301806B816B9E
:10197000C26B8B9291EC33F091EC33F0F1EC34F0DC
:101980006FEC31F0200E3CEC0BF0E8CF2FF50501A9
:101990002F51FF0AD8A4D4EF0CF02F6B200E0C6E41
:1019A0002FC50BF025EC0BF00501010E306F3C0E3E
:1019B000316F250E3CEC0BF0E8CF00F1260E3CEC2D
:1019C0000BF0E8CF01F1270E3CEC0BF0E8CF02F171
:1019D000280E3CEC0BF0E8CF03F1010103AF0BEF55
:1019E0000DF06DEC2EF0250E0C6E00C10BF025EC09
:1019F0000BF0260E0C6E01C10BF025EC0BF0270E40
:101A00000C6E02C10BF025EC0BF0280E0C6E03C11E
:101A10000BF025EC0BF000C157F501C158F502C1E0
:101A200059F503C15AF500C15BF501C15CF502C16E
:101A30005DF503C15EF5290E3CEC0BF0E8CF5FF5D8
:101A4000050160515F5DD8A05FC560F5210E3CECDB
:101A50000BF0E8CF00F1220E3CEC0BF0E8CF01F1E7
:101A6000230E3CEC0BF0E8CF02F1240E3CEC0BF023
:101A7000E8CF03F1010103AF6CEF0DF06DEC2EF038
:101A8000210E0C6E00C10BF025EC0BF0220E0C6E3B
:101A900001C10BF025EC0BF0230E0C6E02C10BF014
:101AA00025EC0BF0240E0C6E03C10BF025EC0BF0B3
:101AB000210E3CEC0BF0E8CF00F1220E3CEC0BF0D9
:101AC000E8CF01F1230E3CEC0BF0E8CF02F1240E3D
:101AD0003CEC0BF0E8CF03F100C161F501C162F508
:101AE00002C163F503C164F5B7EC30F09DEC2FF053
:101AF000F5EC2EF037A0DDEF0DF005012F51020AB5
:101B000016E005012F51030A19E005012F51040ABF
:101B100024E005012F51050A2BE005012F51060A8B
:101B200039E005012F51070A3FE0DDEF0DF0602F8E
:101B3000DAEF0DF05FC560F5DDEF0DF0B0C500F137
:101B400001010F0E001701010051000A36E00101EA
:101B50000051050A32E0DAEF0DF0B0C500F10101E5
:101B60000F0E001701010051000A27E0DAEF0DF017
:101B70000501B051000A21E00501B051150A1DE030
:101B80000501B051300A19E00501B051450A15E0D0
:101B9000DAEF0DF00501B051000A0FE00501B05178
:101BA000300A0BE0DAEF0DF00501B051000A05E054
:101BB000DAEF0DF081BA30EF35F007900001F28EC8
:101BC000F28C12AE03D012BC27EF19F007B0B0EFC1
:101BD0002AF00FB0ACEF23F010BEACEF23F012B838
:101BE000ACEF23F000011650010AD8B426EF1DF027
:101BF00000011650040AD8B438EF1DF003018051DB
:101C000081197F0BD8B4B0EF2AF013EE00F08151A8
:101C10007F0BE126812BE7CFE8FFE00BD8B4B0EFD4
:101C20002AF023EE82F0C2513F0BD926E7CFDFFF27
:101C3000C22BDF50780AD8A4B0EF2AF0078092C1F7
:101C400000F193C101F194C102F195C103F10101C9
:101C5000040E046F000E056F000E066F000E076F76
:101C600072EC2DF000AF3EEF0EF00101030E926F0B
:101C7000000E936F000E946F000E956F030182515A
:101C8000720AD8B488EF23F08251520AD8B488EF90
:101C900023F08251750AD8B488EF23F08251680A84
:101CA000D8B4BCEF0EF08251630AD8B46AEF27F0C3
:101CB0008251690AD8B431EF20F082517A0AD8B43F
:101CC00044EF21F08251490AD8B4D0EF1FF082517D
:101CD000500AD8B4EEEF1EF08251700AD8B431EF3A
:101CE0001FF08251540AD8B45CEF1FF08251740A7D
:101CF000D8B4A2EF1FF08251410AD8B4C1EF0FF05F
:101D000082514B0AD8B4BEEF0EF082516D0AD8B49E
:101D100031EF14F082514D0AD8B44AEF14F08251D9
:101D2000730AD8B4B8EF22F08251530AD8B41DEF29
:101D300023F082514C0AD8B4D9EF14F08251590AD9
:101D4000D8B482EF13F012AE01D0128CA1EF27F0BD
:101D5000040114EE00F080517F0BE12682C4E7FFFE
:101D6000802B120004010D0E826FA8EC0EF00A0EFB
:101D7000826FA8EC0EF012009FEF27F004014B0ECB
:101D8000826FA8EC0EF004012C0E826FA8EC0EF00E
:101D900081B802D036B630D003018351430AD8B49B
:101DA00003EF0FF003018351630AD8B405EF0FF07E
:101DB00003018351520AD8B407EF0FF00301835196
:101DC000720AD8B409EF0FF003018351470AD8B45F
:101DD0000BEF0FF003018351670AD8B40DEF0FF03A
:101DE00003018351540AD8B40FEF0FF0030183515C
:101DF000740AD8B47FEF0FF003018351550AD8B4A9
:101E000011EF0FF083D036807BD0369079D03682B8
:101E100077D0369275D0368473D0369471D03686AA
:101E20006FD084C330F185C331F186C332F187C3EB
:101E300033F10101296BBBEC2EF032EC2EF000C126
:101E400004F101C105F102C106F103C107F1AEECD5
:101E50002EF0200EF86EF76AF66A0900F5CF2CF125
:101E60000900F5CF2DF10900F5CF2EF10900F5CFCE
:101E70002FF10900F5CF30F10900F5CF31F109005C
:101E8000F5CF32F10900F5CF33F10101296BBBEC3D
:101E90002EF032EC2EF072EC2DF00101006758EFBD
:101EA0000FF0016758EF0FF0026758EF0FF003676C
:101EB00001D025D004014E0E826FA8EC0EF0040173
:101EC0006F0E826FA8EC0EF004014D0E826FA8EC2D
:101ED0000EF00401610E826FA8EC0EF00401740E86
:101EE000826FA8EC0EF00401630E826FA8EC0EF076
:101EF0000401680E826FA8EC0EF09FEF27F0369673
:101F0000CD0E0C6E36C00BF025EC0BF0CD0E3CEC7C
:101F10000BF0E8CF36F036B006D00401630E826FC6
:101F2000A8EC0EF005D00401430E826FA8EC0EF071
:101F300036B206D00401720E826FA8EC0EF005D006
:101F40000401520E826FA8EC0EF036B406D00401E4
:101F5000670E826FA8EC0EF005D00401470E826F69
:101F6000A8EC0EF036B606D00401740E826FA8EC11
:101F70000EF005D00401540E826FA8EC0EF09FEF16
:101F800027F00401410E826FA8EC0EF0030183518B
:101F9000310AD8B4A2EF12F003018351320AD8B447
:101FA000D2EF11F003018351330AD8B45BEF11F083
:101FB00003018351340AD8B44BEF10F0030183516D
:101FC000350AD8B4EBEF0FF004013F0E826FA8EC96
:101FD0000EF09FEF27F003018451300AD8B411EFBF
:101FE00010F003018451310AD8B414EF10F003014A
:101FF0008451650AD8B405EF10F003018451640AD6
:10200000D8B408EF10F015EF10F0388009EF10F099
:102010003890FB0E0C6E38C00BF025EC0BF015EF72
:1020200010F08B9015EF10F08B800401350E826F4D
:10203000A8EC0EF004012C0E826FA8EC0EF08BB011
:1020400029EF10F00401300E826FA8EC0EF02EEF95
:1020500010F00401310E826FA8EC0EF004012C0E7A
:10206000826FA8EC0EF0FB0E3CEC0BF0E8CF38F0E2
:1020700038B042EF10F00401640E826FA8EC0EF04D
:1020800047EF10F00401650E826FA8EC0EF049EFE7
:1020900010F09FEF27F0CC0E3CEC0BF0E8CF0BF0EC
:1020A00004012C0E826FA8EC0EF003018451310A5A
:1020B000D8B46FEF10F003018451300AD8B471EF37
:1020C00010F0030184514D0AD8B47BEF10F00301E6
:1020D0008451540AD8B482EF10F099EF10F08A843A
:1020E00001D08A940BAE04D00BAC02D00BBA21D035
:1020F000E00E0B1218D01F0E0B168539E844E00BCA
:102100000B1211D0E00E0B16AEEC2EF085C332F19F
:1021100086C333F10101296BBBEC2EF032EC2EF0BB
:1021200000511F0B0B12CC0E0C6E0BC00BF025ECEC
:102130000BF00401340E826FA8EC0EF004012C0E9B
:10214000826FA8EC0EF0CC0E3CEC0BF0E8CF1DF04B
:102150008AB406D00401300E826FA8EC0EF005D0D0
:102160000401310E826FA8EC0EF004012C0E826F78
:10217000A8EC0EF01D38E840070BE8CF82F404010C
:10218000300E8227A8EC0EF004012C0E826FA8EC12
:102190000EF06DEC2EF01D501F0BE8CF00F110EC8F
:1021A0002EF032C182F40401300E8227A8EC0EF02A
:1021B00033C182F40401300E8227A8EC0EF0040132
:1021C0002C0E826FA8EC0EF06DEC2EF030C000F1FA
:1021D00000AF0BD0FF0E016FFF0E026FFF0E036FFB
:1021E00004012D0E826FA8EC0EF010EC2EF031C120
:1021F00082F40401300E8227A8EC0EF032C182F482
:102200000401300E8227A8EC0EF033C182F40401E1
:10221000300E8227A8EC0EF004012C0E826FA8EC81
:102220000EF06DEC2EF02FC000F110EC2EF031C14D
:1022300082F40401300E8227A8EC0EF032C182F441
:102240000401300E8227A8EC0EF033C182F40401A1
:10225000300E8227A8EC0EF004012C0E826FA8EC41
:102260000EF06DEC2EF031C000F100AF0BD0FF0E80
:10227000016FFF0E026FFF0E036F04012D0E826FC0
:10228000A8EC0EF010EC2EF031C182F40401300EF7
:102290008227A8EC0EF032C182F40401300E8227AE
:1022A000A8EC0EF033C182F40401300E8227A8ECB2
:1022B0000EF09FEF27F0CB0E3CEC0BF0E8CF0BF0CD
:1022C00004012C0E826FA8EC0EF003018451450A24
:1022D000D8B47FEF11F003018451440AD8B482EFDF
:1022E00011F003018451300AD8B485EF11F00301D5
:1022F0008451310AD8B489EF11F094EF11F00B9E9C
:102300008EEF11F00B8E8EEF11F0FC0E0B168EEF90
:1023100011F0FC0E0B160B808EEF11F0CB0E0C6E35
:102320000BC00BF025EC0BF00401330E826FA8EC10
:102330000EF004012C0E826FA8EC0EF0CB0E3CECDC
:102340000BF0E8CF1CF01CBEADEF11F00401450E00
:10235000826FA8EC0EF0B2EF11F00401440E826F10
:10236000A8EC0EF004012C0E826FA8EC0EF0040114
:10237000300E826FA8EC0EF004012C0E826FA8ECD8
:102380000EF01CB0CBEF11F00401300E826FA8EC00
:102390000EF0D0EF11F00401310E826FA8EC0EF0B8
:1023A0009FEF27F0CA0E3CEC0BF0E8CF0BF00401D6
:1023B0002C0E826FA8EC0EF003018451450AD8B4AC
:1023C0000EEF12F003018451440AD8B411EF12F059
:1023D000030184514D0AD8B41AEF12F0030184515D
:1023E000410AD8B414EF12F003018451460AD8B45C
:1023F00017EF12F003018451560AD8B422EF12F0FD
:1024000003018451500AD8B42DEF12F00301845116
:10241000520AD8B430EF12F039EF12F00B9E33EFBE
:1024200012F00B8E33EF12F00B9C33EF12F00B8C8B
:1024300033EF12F0FC0E0B1685C3E8FF030B0B12F3
:1024400033EF12F0C70E0B1685C3E8FF070BE84603
:10245000E846E8460B1233EF12F00B8433EF12F02C
:102460000B9433EF12F0CA0E0C6E0BC00BF025EC80
:102470000BF0CA0E3CEC0BF0E8CF1BF00401320E5F
:10248000826FA8EC0EF004012C0E826FA8EC0EF007
:102490001BBE52EF12F00401450E826FA8EC0EF045
:1024A00057EF12F00401440E826FA8EC0EF0040105
:1024B0002C0E826FA8EC0EF01BC0E8FF030BE8CFD8
:1024C00082F40401300E8227A8EC0EF004012C0ED9
:1024D000826FA8EC0EF01BBC75EF12F00401410EE8
:1024E000826FA8EC0EF07AEF12F00401460E826FB4
:1024F000A8EC0EF004012C0E826FA8EC0EF01BC0AD
:10250000E8FF380BE842E842E842E8CF82F40401F1
:10251000300E8227A8EC0EF004012C0E826FA8EC7E
:102520000EF01BB49BEF12F00401520E826FA8EC68
:102530000EF0A0EF12F00401500E826FA8EC0EF026
:102540009FEF27F0C90E3CEC0BF0E8CF0BF0040135
:102550002C0E826FA8EC0EF003018451450AD8B40A
:10256000C0EF12F003018451440AD8B4C3EF12F053
:10257000030184514D0AD8B4C6EF12F0D4EF12F023
:102580000B9ECEEF12F00B8ECEEF12F0F80E0B1664
:1025900085C3E8FF070B0B12CEEF12F0C90E0C6ECD
:1025A0000BC00BF025EC0BF00401310E826FA8EC90
:1025B0000EF004012C0E826FA8EC0EF0C90E3CEC5C
:1025C0000BF0E8CF1AF01ABE06D00401450E826F58
:1025D000A8EC0EF005D00401440E826FA8EC0EF0BA
:1025E00004012C0E826FA8EC0EF01AC0E8FF070B56
:1025F000E8CF82F40401300E8227A8EC0EF004012B
:102600002C0E826FA8EC0EF007806DEC2EF02BC024
:10261000E8FF003B00430043030B10EC2EF033C1F6
:1026200082F40401300E8227A8EC0EF004012C0E77
:10263000826FA8EC0EF06DEC2EF02BC001F1019F23
:10264000019D2CC000F1010110EC2EF02FC182F48D
:102650000401300E8227A8EC0EF030C182F4040190
:10266000300E8227A8EC0EF031C182F40401300E46
:102670008227A8EC0EF032C182F40401300E8227CA
:10268000A8EC0EF033C182F40401300E8227A8ECCE
:102690000EF004012C0E826FA8EC0EF06DEC2EF003
:1026A0002DC001F12EC000F1D89001330033D89035
:1026B00001330033010110EC2EF02FC182F404012C
:1026C000300E8227A8EC0EF030C182F40401300EE7
:1026D0008227A8EC0EF031C182F40401300E82276B
:1026E000A8EC0EF032C182F40401300E8227A8EC6F
:1026F0000EF033C182F40401300E8227A8EC0EF0F4
:102700009FEF27F0FC0E3CEC0BF0E8CF0BF0030141
:102710008351520AD8B4B9EF13F003018351720AFE
:10272000D8B4BCEF13F003018351500AD8B4BFEF03
:1027300013F003018351700AD8B4C2EF13F0030100
:102740008351550AD8B4C5EF13F003018351750ABC
:10275000D8B4C8EF13F003018351430AD8B4D1EFC2
:1027600013F003018351630AD8B4D4EF13F0DDEF03
:1027700013F00B90D7EF13F00B80D7EF13F00B9201
:10278000D7EF13F00B82D7EF13F00B94D7EF13F0C2
:102790000B84D7EF13F00B96D7EF13F00B86D7EF20
:1027A00013F00B98D7EF13F00B88D7EF13F0FC0E54
:1027B0000C6E0BC00BF025EC0BF00401590E826F70
:1027C000A8EC0EF01190119211941198FC0E3CECB3
:1027D0000BF0E8CF0BF00BA011800BA211820BA421
:1027E00011840BA8118811A0FDEF13F00401520E03
:1027F000826FA8EC0EF002EF14F00401720E826FEB
:10280000A8EC0EF011A80CEF14F00401430E826F37
:10281000A8EC0EF011EF14F00401630E826FA8EC27
:102820000EF011A21BEF14F00401500E826FA8EC01
:102830000EF020EF14F00401700E826FA8EC0EF081
:1028400011A42AEF14F00401550E826FA8EC0EF0CB
:102850002FEF14F00401750E826FA8EC0EF09FEFBD
:1028600027F004016D0E826FA8EC0EF00301835176
:10287000300AD8B489EF14F003018351310AD8B477
:102880009CEF14F003018351320AD8B4AFEF14F077
:10289000A1EF27F004014D0E826FA8EC0EF0AEEC14
:1028A0002EF084C331F185C332F186C333F10101C7
:1028B000296BBBEC2EF032EC2EF003018351300A71
:1028C000D8B471EF14F003018351310AD8B479EF11
:1028D00014F003018351320AD8B481EF14F0A1EF50
:1028E00027F0FD0E0C6E00C10BF025EC0BF089EF0C
:1028F00014F0FE0E0C6E00C10BF025EC0BF09CEFFB
:1029000014F0FF0E0C6E00C10BF025EC0BF0AFEFD6
:1029100014F00401300E826FA8EC0EF004012C0EAE
:10292000826FA8EC0EF06DEC2EF0FD0E3CEC0BF07F
:10293000E8CF00F1C0EF14F00401310E826FA8EC73
:102940000EF004012C0E826FA8EC0EF06DEC2EF050
:10295000FE0E3CEC0BF0E8CF00F1C0EF14F00401E8
:10296000320E826FA8EC0EF06DEC2EF004012C0EEE
:10297000826FA8EC0EF0FF0E3CEC0BF0E8CF00F1FC
:1029800010EC2EF031C182F40401300E8227A8EC45
:102990000EF032C182F40401300E8227A8EC0EF052
:1029A00033C182F40401300E8227A8EC0EF09FEFB1
:1029B00027F003018351300AD8B4D4EF19F0030192
:1029C0008351310AD8B401EF1BF003018351320A5D
:1029D000D8B46FEF1BF003018351330AD8B47FEFF3
:1029E0001BF003018351340AD8B48FEF1BF00301AD
:1029F0008351350AD8B43FEF1DF003018351360AE5
:102A0000D8B46DEF1DF003018351370AD8B4ACEF91
:102A100017F003018351380AD8B44AEF18F00301C4
:102A20008351460AD8B47FEF1CF0030183514D0A4D
:102A3000D8B425EF16F0030183516D0AD8B43FEFE7
:102A400016F0030183515A0AD8B47BEF1AF0030140
:102A50008351490AD8B46DEF1EF003018351500A27
:102A6000D8B49FEF1DF003018351540AD8B418EF76
:102A70001EF003018351630AD8B45FEF16F003011F
:102A80008351430AD8B457EF17F003018351730AF7
:102A9000D8B45DEF16F003018351610AD8B472EF28
:102AA00015F003018351650AD8B424EF1AF003012D
:102AB0008351450AD8B432EF1AF003018351620AF8
:102AC000D8B440EF1AF003018351420AD8B44EEF54
:102AD0001AF003018351760AD8B45CEF1AF0D8A437
:102AE000A1EF27F004014C0E826FA8EC0EF0040158
:102AF000610E826FA8EC0EF09DEC2FF004012C0EFD
:102B0000826FA8EC0EF06DEC2EF0AFC500F1010164
:102B100010EC2EF031C182F40401300E8227A8ECB3
:102B20000EF032C182F40401300E8227A8EC0EF0C0
:102B300033C182F40401300E8227A8EC0EF00401A8
:102B40002C0E826FA8EC0EF06DEC2EF0B0C500F1EB
:102B5000010110EC2EF031C182F40401300E822705
:102B6000A8EC0EF032C182F40401300E8227A8ECEA
:102B70000EF033C182F40401300E8227A8EC0EF06F
:102B800004012C0E826FA8EC0EF06DEC2EF0B1C596
:102B900000F1010110EC2EF031C182F40401300E7D
:102BA0008227A8EC0EF032C182F40401300E822795
:102BB000A8EC0EF033C182F40401300E8227A8EC99
:102BC0000EF004012C0E826FA8EC0EF06DEC2EF0CE
:102BD000B2C500F1010110EC2EF031C182F4040104
:102BE000300E8227A8EC0EF032C182F40401300EC0
:102BF0008227A8EC0EF033C182F40401300E822744
:102C0000A8EC0EF004012C0E826FA8EC0EF06DEC17
:102C10002EF0B6C500F1010110EC2EF031C182F4A6
:102C20000401300E8227A8EC0EF032C182F40401B8
:102C3000300E8227A8EC0EF033C182F40401300E6E
:102C40008227A8EC0EF09BEF1DF0AEEC2EF084C3B3
:102C500033F1BBEC2EF032EC2EF0200E0C6E00C1E6
:102C60000BF025EC0BF000C12FF505012F51000AE8
:102C700006E005012F51010A02E037EC30F00401B3
:102C80004C0E826FA8EC0EF004014D0E826FA8EC82
:102C90000EF004012C0E826FA8EC0EF06DEC2EF0FD
:102CA0002FC500F110EC2EF033C182F40401300E78
:102CB0008227A8EC0EF09BEF1DF030EF35F00401F9
:102CC0004C0E826FA8EC0EF00401630E826FA8EC2C
:102CD0000EF0F5EC2EF004012C0E826FA8EC0EF035
:102CE00074EC16F09BEF1DF06DEC2EF0B5C500F105
:102CF0000101003B0F0E001710EC2EF033C182F4DF
:102D00000401300E8227A8EC0EF0B5C500F10101D8
:102D10000F0E0101001710EC2EF033C182F40401F4
:102D2000300E8227A8EC0EF004012D0E826FA8EC65
:102D30000EF0B4C500F10101003B0F0E001710ECBE
:102D40002EF033C182F40401300E8227A8EC0EF07D
:102D5000B4C500F101010F0E0101001710EC2EF0B7
:102D600033C182F40401300E8227A8EC0EF0040176
:102D70002D0E826FA8EC0EF0B3C500F10101003BEF
:102D80000F0E001710EC2EF033C182F40401300E48
:102D90008227A8EC0EF0B3C500F101010F0E01016E
:102DA000001710EC2EF033C182F40401300E82279C
:102DB000A8EC0EF00401200E826FA8EC0EF0B2C554
:102DC00000F10F0E0101001710EC2EF033C182F458
:102DD0000401300E8227A8EC0EF00401200E826F51
:102DE000A8EC0EF0B1C500F101010101003B0F0E8E
:102DF000001710EC2EF033C182F40401300E82274C
:102E0000A8EC0EF0B1C500F101010F0E0101001791
:102E100010EC2EF033C182F40401300E8227A8ECAE
:102E20000EF004013A0E826FA8EC0EF0B0C500F16E
:102E30000101003B0F0E001710EC2EF033C182F49D
:102E40000401300E8227A8EC0EF0B0C500F101019C
:102E50000F0E0101001710EC2EF033C182F40401B3
:102E6000300E8227A8EC0EF004013A0E826FA8EC17
:102E70000EF0AFC500F10101003B0F0E001710EC82
:102E80002EF033C182F40401300E8227A8EC0EF03C
:102E9000AFC500F101010F0E001710EC2EF033C189
:102EA00082F40401300E8227A8EC0EF0120084C3D5
:102EB000E8FF0F0BE83AE8CFB5F585C3E8FF0F0B45
:102EC0000501B51387C3E8FF0F0BE83AE8CFB4F567
:102ED00088C3E8FF0F0B0501B4138AC3E8FF0F0B8B
:102EE000E83AE8CFB3F58BC3E8FF0F0B0501B31346
:102EF0008DC3E8FF0F0BE8CFB2F58FC3E8FF0F0BD0
:102F0000E83AE8CFB1F590C3E8FF0F0B0501B11324
:102F100092C3E8FF0F0BE83AE8CFB0F593C3E8FFA0
:102F20000F0B0501B01395C3E8FF0F0BE83AE8CF8C
:102F3000AFF596C3E8FF0F0B0501AF1350EC2FF070
:102F400004014C0E826FA8EC0EF00401430E826F58
:102F5000A8EC0EF069EF16F0078404014C0E826FA6
:102F6000A8EC0EF00401370E826FA8EC0EF00401FD
:102F70002C0E826FA8EC0EF005012E51130A06E00C
:102F800005012E51170A0DE047EF18F00101000E60
:102F9000006F000E016F100E026F000E036FDAEF6C
:102FA00017F00101000E006F000E016F000E026F9E
:102FB000010E036F10EC2EF02AC182F40401300ED2
:102FC0008227A8EC0EF02BC182F40401300E822778
:102FD000A8EC0EF02CC182F40401300E8227A8EC7C
:102FE0000EF02DC182F40401300E8227A8EC0EF001
:102FF0002EC182F40401300E8227A8EC0EF02FC1FE
:1030000082F40401300E8227A8EC0EF030C182F465
:103010000401300E8227A8EC0EF031C182F40401C5
:10302000300E8227A8EC0EF032C182F40401300E7B
:103030008227A8EC0EF033C182F40401300E8227FF
:10304000A8EC0EF004012C0E826FA8EC0EF001012A
:10305000100E006F000E016F000E026F000E036F66
:1030600010EC2EF031C182F40401300E8227A8EC5E
:103070000EF032C182F40401300E8227A8EC0EF06B
:1030800033C182F40401300E8227A8EC0EF00794BD
:103090009BEF1DF00501216B226B236B246B040158
:1030A0004C0E826FA8EC0EF00401380E826FA8EC73
:1030B0000EF004012C0E826FA8EC0EF00101100E30
:1030C000006F000E016F000E026F000E036F10EC18
:1030D0002EF02AC182F40401300E8227A8EC0EF0F3
:1030E0002BC182F40401300E8227A8EC0EF02CC113
:1030F00082F40401300E8227A8EC0EF02DC182F478
:103100000401300E8227A8EC0EF02EC182F40401D7
:10311000300E8227A8EC0EF02FC182F40401300E8D
:103120008227A8EC0EF030C182F40401300E822711
:10313000A8EC0EF031C182F40401300E8227A8EC15
:103140000EF032C182F40401300E8227A8EC0EF09A
:1031500033C182F40401300E8227A8EC0EF0040182
:103160002C0E826FA8EC0EF025C500F126C501F1EA
:1031700027C502F128C503F10101100E046F000EEE
:10318000056F000E066F000E076FA3EC2DF000C157
:1031900033F501C134F502C135F503C136F510EC44
:1031A0002EF02AC182F40401300E8227A8EC0EF022
:1031B0002BC182F40401300E8227A8EC0EF02CC142
:1031C00082F40401300E8227A8EC0EF02DC182F4A7
:1031D0000401300E8227A8EC0EF02EC182F4040107
:1031E000300E8227A8EC0EF02FC182F40401300EBD
:1031F0008227A8EC0EF030C182F40401300E822741
:10320000A8EC0EF031C182F40401300E8227A8EC44
:103210000EF032C182F40401300E8227A8EC0EF0C9
:1032200033C182F40401300E8227A8EC0EF0B2EC18
:103230000EF00501336724EF19F0346724EF19F01D
:10324000356724EF19F0366702D0C3EF19F0129EEC
:10325000129C21C500F122C501F123C502F124C54C
:1032600003F1899A400EC76E200EC66E9E96C69ECA
:103270000B0EC96EFF0E9EB602D0E82EFCD79E96AE
:10328000C69E02C1C9FFFF0E9EB602D0E82EFCD733
:103290009E96C69E01C1C9FFFF0E9EB602D0E82EC3
:1032A000FCD79E96C69E00C1C9FFFF0E9EB602D0F7
:1032B000E82EFCD79E96C69EC952FF0E9EB602D03F
:1032C000E82EFCD70501100E326F040114EE00F059
:1032D00080517F0BE1269E96C69EC952FF0E9EB678
:1032E00002D0E82EFCD7C9CFE7FF0401802B0501EF
:1032F000322F65EF19F0898A33C500F134C501F129
:1033000035C502F136C503F10101010E046F000E4F
:10331000056F000E066F000E076F72EC2DF000C1F6
:1033200033F501C134F502C135F503C136F50501A8
:103330003367A2EF19F03467A2EF19F03567A2EFF7
:1033400019F0366702D0C3EF19F021C500F122C58C
:1033500001F123C502F124C503F10101100E046F30
:10336000000E056F000E066F000E076F77EC2DF054
:1033700000C121F501C122F502C123F503C124F5E5
:10338000128EA1EF27F00401450E826FA8EC0EF01B
:1033900004014F0E826FA8EC0EF00401460E826FFE
:1033A000A8EC0EF09BEF1DF00784F1EC34F06DEC0F
:1033B0002EF02DC500F110EC2EF004014C0E826FA2
:1033C000A8EC0EF00401300E826FA8EC0EF00401A0
:1033D0002C0E826FA8EC0EF031C182F40401300E85
:1033E0008227A8EC0EF032C182F40401300E82274D
:1033F000A8EC0EF033C182F40401300E8227A8EC51
:103400000EF004012C0E826FA8EC0EF06DEC2EF085
:103410002EC500F110EC2EF031C182F40401300E03
:103420008227A8EC0EF032C182F40401300E82270C
:10343000A8EC0EF033C182F40401300E8227A8EC10
:103440000EF007949BEF1DF004014C0E826FA8EC68
:103450000EF00401650E826FA8EC0EF013EC31F053
:103460009BEF1DF004014C0E826FA8EC0EF00401DE
:10347000450E826FA8EC0EF02AEC31F09BEF1DF0A8
:1034800004014C0E826FA8EC0EF00401620E826FF4
:10349000A8EC0EF058EC31F09BEF1DF004014C0E3F
:1034A000826FA8EC0EF00401420E826FA8EC0EF0C1
:1034B00041EC31F09BEF1DF004014C0E826FA8EC43
:1034C0000EF00401760E826FA8EC0EF004012C0EB3
:1034D000826FA8EC0EF010A807D00401310E826FA5
:1034E000A8EC0EF09BEF1DF00401300E826FA8ECEB
:1034F0000EF09BEF1DF004014C0E826FA8EC0EF055
:1035000004015A0E826FA8EC0EF004012C0E826F9B
:10351000A8EC0EF0F1EC34F06DEC2EF005012E511C
:10352000130A06E005012E51170A0DE0ACEF1AF060
:103530000101000E006F000E016F100E026F000EF1
:10354000036FACEF1AF00101000E006F000E016F67
:10355000000E026F010E036F0101100E046F000ECA
:10356000056F000E066F000E076FA3EC2DF010EC38
:103570002EF02AC182F40401300E8227A8EC0EF04E
:103580002BC182F40401300E8227A8EC0EF02CC16E
:1035900082F40401300E8227A8EC0EF02DC182F4D3
:1035A0000401300E8227A8EC0EF02EC182F4040133
:1035B000300E8227A8EC0EF02FC182F40401300EE9
:1035C0008227A8EC0EF030C182F40401300E82276D
:1035D000A8EC0EF031C182F40401300E8227A8EC71
:1035E0000EF032C182F40401300E8227A8EC0EF0F6
:1035F00033C182F40401300E8227A8EC0EF09BEF59
:103600001DF0078404014C0E826FA8EC0EF004013B
:10361000310E826FA8EC0EF004012C0E826FA8EC24
:103620000EF025C500F126C501F127C502F128C518
:1036300003F10101100E046F000E056F000E066FFE
:10364000000E076FA3EC2DF010EC2EF02AC182F4CF
:103650000401300E8227A8EC0EF02BC182F4040185
:10366000300E8227A8EC0EF02CC182F40401300E3B
:103670008227A8EC0EF02DC182F40401300E8227BF
:10368000A8EC0EF02EC182F40401300E8227A8ECC3
:103690000EF02FC182F40401300E8227A8EC0EF048
:1036A00030C182F40401300E8227A8EC0EF031C143
:1036B00082F40401300E8227A8EC0EF032C182F4AD
:1036C0000401300E8227A8EC0EF033C182F404010D
:1036D000300E8227A8EC0EF007949BEF1DF00784B4
:1036E00004014C0E826FA8EC0EF00401320E826FC2
:1036F000A8EC0EF047EC33F007949BEF1DF0078425
:1037000004014C0E826FA8EC0EF00401330E826FA0
:10371000A8EC0EF0A4EC33F007940CEF1BF0078438
:1037200004014C0E826FA8EC0EF00401340E826F7F
:10373000A8EC0EF004012C0E826FA8EC0EF0AEEC9B
:103740002EF084C32AF185C32BF186C32CF187C3E5
:103750002DF188C32EF189C32FF18AC330F18BC3B9
:1037600031F18CC332F18DC333F10101296BBBEC14
:103770002EF032EC2EF0100E046F000E056F000ECE
:10378000066F000E076F83EC2DF000C121F501C11B
:1037900022F502C123F503C124F5A4EC34F038C5A9
:1037A000AFF539C5B0F53AC5B1F53BC5B2F53CC585
:1037B000B3F53DC5B4F53EC5B5F574EC16F004019E
:1037C0002C0E826FA8EC0EF03FC500F140C501F150
:1037D00041C502F142C503F10101000E046F000E64
:1037E000056F010E066F000E076FA3EC2DF010ECB5
:1037F0002EF02967FEEF1BF003EF1CF004012D0EE5
:10380000826FA8EC0EF030C182F40401300E8227E2
:10381000A8EC0EF031C182F40401300E8227A8EC2E
:103820000EF004012E0E826FA8EC0EF032C182F46D
:103830000401300E8227A8EC0EF033C182F404019B
:10384000300E8227A8EC0EF004012C0E826FA8EC3B
:103850000EF06DEC2EF043C500F144C501F1CBEC48
:1038600028F004012C0E826FA8EC0EF06DEC2EF007
:1038700045C500F110EC2EF031C182F40401300E88
:103880008227A8EC0EF032C182F40401300E8227A8
:10389000A8EC0EF033C182F40401300E8227A8ECAC
:1038A0000EF004012C0E826FA8EC0EF037C5E8FF75
:1038B000E8B806D00401300E826FA8EC0EF005D0F7
:1038C0000401310E826FA8EC0EF038A07CEF1CF0E2
:1038D00004012C0E826FA8EC0EF037C5E8FFE8BAA1
:1038E00006D00401300E826FA8EC0EF005D0040162
:1038F000310E826FA8EC0EF007949BEF1DF0AEEC3A
:103900002EF085C32AF186C32BF187C32CF188C31F
:103910002DF189C32EF18AC32FF18BC330F18CC3F3
:1039200031F18DC332F18EC333F10101296BBBEC50
:103930002EF032EC2EF00101010E046F000E056F27
:10394000000E066F000E076F72EC2DF0100E046F64
:10395000000E056F000E066F000E076F83EC2DF052
:1039600000C129F501C12AF502C12BF503C12CF5CF
:10397000CEEC32F004014C0E826FA8EC0EF0040184
:10398000460E826FA8EC0EF004012C0E826FA8EC9C
:103990000EF025C500F126C501F127C502F128C5A5
:1039A00003F10101100E046F000E056F000E066F8B
:1039B000000E076FA3EC2DF010EC2EF02AC182F45C
:1039C0000401300E8227A8EC0EF02BC182F4040112
:1039D000300E8227A8EC0EF02CC182F40401300EC8
:1039E0008227A8EC0EF02DC182F40401300E82274C
:1039F000A8EC0EF02EC182F40401300E8227A8EC50
:103A00000EF02FC182F40401300E8227A8EC0EF0D4
:103A100030C182F40401300E8227A8EC0EF031C1CF
:103A200082F40401300E8227A8EC0EF032C182F439
:103A30000401300E8227A8EC0EF033C182F4040199
:103A4000300E8227A8EC0EF09BEF1DF0A4EC33F0B3
:103A500038A033EF1DF08B800F9A0F9C0F9E030E42
:103A6000166EA1EF27F0050E166E3780A1EF27F036
:103A7000A4EC33F0050E166E3780A1EF27F0040199
:103A80004C0E826FA8EC0EF00401350E826FA8EC8C
:103A90000EF004012C0E826FA8EC0EF06DEC2EF0EF
:103AA0000784B9C500F1079410EC2EF031C182F4FF
:103AB0000401300E8227A8EC0EF032C182F404011A
:103AC000300E8227A8EC0EF033C182F40401300ED0
:103AD0008227A8EC0EF09BEF1DF067EC33F06DEC45
:103AE0002EF037C500F110EC2EF004014C0E826F61
:103AF000A8EC0EF00401360E826FA8EC0EF0040163
:103B00002C0E826FA8EC0EF031C182F40401300E4D
:103B10008227A8EC0EF032C182F40401300E822715
:103B2000A8EC0EF033C182F40401300E8227A8EC19
:103B30000EF09BEF1DF0B2EC0EF0A1EF27F00401A8
:103B40004C0E826FA8EC0EF00401500E826FA8ECB0
:103B50000EF004012C0E826FA8EC0EF085C32AF142
:103B600086C32BF187C32CF188C32DF189C32EF1B5
:103B70008AC32FF18BC330F18CC331F18DC332F185
:103B80008EC333F10101BBEC2EF032EC2EF00301B9
:103B90008451530A0DE0030184514D0A38E00401B9
:103BA000780E826FA8EC0EF0B2EC0EF0A1EF27F0C9
:103BB0000401530E826FA8EC0EF0250E0C6E00C1AE
:103BC0000BF025EC0BF0260E0C6E01C10BF025EC72
:103BD0000BF0270E0C6E02C10BF025EC0BF0280E3B
:103BE0000C6E03C10BF025EC0BF000C157F501C1C1
:103BF00058F502C159F503C15AF500C15BF501C181
:103C00005CF502C15DF503C15EF57CEF1EF00401B9
:103C10004D0E826FA8EC0EF0290E0C6E00C10BF059
:103C200025EC0BF000C15FF500C160F57CEF1EF0E4
:103C300004014C0E826FA8EC0EF00401540E826F4A
:103C4000A8EC0EF004012C0E826FA8EC0EF084C3D9
:103C50002AF185C32BF186C32CF187C32DF188C3CC
:103C60002EF189C32FF18AC330F18BC331F18DC39B
:103C700032F18EC333F10101BBEC2EF032EC2EF0A9
:103C80000101000E046F000E056F010E066F000E9D
:103C9000076F83EC2DF0210E0C6E00C10BF025ECAC
:103CA0000BF0220E0C6E01C10BF025EC0BF0230E75
:103CB0000C6E02C10BF025EC0BF0240E0C6E03C150
:103CC0000BF025EC0BF000C161F501C162F502C1FA
:103CD00063F503C164F57CEF1EF004014C0E826FA6
:103CE000A8EC0EF00401490E826FA8EC0EF004015E
:103CF0002C0E826FA8EC0EF0250E3CEC0BF0E8CFFA
:103D000000F1260E3CEC0BF0E8CF01F1270E3CEC65
:103D10000BF0E8CF02F1280E3CEC0BF0E8CF03F1FA
:103D200010EC2EF0D3EC2BF00401730E826FA8EC94
:103D30000EF004012C0E826FA8EC0EF06DEC2EF04C
:103D4000290E3CEC0BF0E8CF00F110EC2EF0D3EC98
:103D50002BF004016D0E826FA8EC0EF004012C0E06
:103D6000826FA8EC0EF05BC500F15CC501F15DC58A
:103D700002F15EC503F110EC2EF0D3EC2BF0040140
:103D8000730E826FA8EC0EF004012C0E826FA8EC6B
:103D90000EF06DEC2EF060C500F110EC2EF0D3ECBF
:103DA0002BF004016D0E826FA8EC0EF004012C0EB6
:103DB000826FA8EC0EF061C500F162C501F163C528
:103DC00002F164C503F1BCEC27F004012C0E826FF4
:103DD000A8EC0EF0B2EC0EF0A1EF27F083C32AF1AD
:103DE00084C32BF185C32CF186C32DF187C32EF13B
:103DF00088C32FF189C330F18AC331F18BC332F10B
:103E00008CC333F10101BBEC2EF032EC2EF0160E18
:103E10000C6E00C10BF025EC0BF0170E0C6E01C1FF
:103E20000BF025EC0BF0180E0C6E02C10BF025EC1C
:103E30000BF0190E0C6E03C10BF025EC0BF000C15A
:103E40008EF101C18FF102C190F103C191F100C166
:103E500092F101C193F102C194F103C195F1D0EF48
:103E60001FF083C32AF184C32BF185C32CF186C3D1
:103E70002DF187C32EF188C32FF189C330F18AC396
:103E800031F18BC332F18CC333F10101BBEC2EF065
:103E900032EC2EF000C18EF101C18FF102C190F120
:103EA00003C191F100C192F101C193F102C194F1FA
:103EB00003C195F1D0EF1FF083C32AF184C32BF126
:103EC00085C32CF186C32DF187C32EF188C32FF152
:103ED00089C330F18AC331F18CC332F18DC333F120
:103EE0000101BBEC2EF032EC2EF00101000E046F4C
:103EF000000E056F010E066F000E076F83EC2DF0AC
:103F00001A0E0C6E00C10BF025EC0BF01B0E0C6EA4
:103F100001C10BF025EC0BF01C0E0C6E02C10BF076
:103F200025EC0BF01D0E0C6E03C10BF025EC0BF015
:103F300000C196F101C197F102C198F103C199F155
:103F4000D0EF1FF083C32AF184C32BF185C32CF17A
:103F500086C32DF187C32EF188C32FF189C330F1B9
:103F60008AC331F18CC332F18DC333F10101BBEC53
:103F70002EF032EC2EF00101000E046F000E056FE2
:103F8000010E066F000E076F83EC2DF000C196F155
:103F900001C197F102C198F103C199F1D0EF1FF06F
:103FA000160E3CEC0BF0E8CF00F1170E3CEC0BF0DA
:103FB000E8CF01F1180E3CEC0BF0E8CF02F1190E3E
:103FC0003CEC0BF0E8CF03F110EC2EF0D3EC2BF02F
:103FD0000401730E826FA8EC0EF004012C0E826FA8
:103FE000A8EC0EF08EC100F18FC101F190C102F179
:103FF00091C103F110EC2EF0D3EC2BF00401730E01
:10400000826FA8EC0EF004012C0E826FA8EC0EF06B
:104010001A0E3CEC0BF0E8CF00F11B0E3CEC0BF061
:10402000E8CF01F11C0E3CEC0BF0E8CF02F11D0EC5
:104030003CEC0BF0E8CF03F1BCEC27F004012C0EB4
:10404000826FA8EC0EF096C100F197C101F198C102
:1040500002F199C103F1BCEC27F0B2EC0EF0A1EF34
:1040600027F00401690E826FA8EC0EF004012C0EFB
:10407000826FA8EC0EF00101040E006F000E016FBC
:10408000000E026F000E036F10EC2EF02CC182F4B4
:104090000401300E8227A8EC0EF02DC182F4040139
:1040A000300E8227A8EC0EF02EC182F40401300EEF
:1040B0008227A8EC0EF02FC182F40401300E822773
:1040C000A8EC0EF030C182F40401300E8227A8EC77
:1040D0000EF031C182F40401300E8227A8EC0EF0FC
:1040E00032C182F40401300E8227A8EC0EF033C1F5
:1040F00082F40401300E8227A8EC0EF004012C0E8D
:10410000826FA8EC0EF00101060E006F000E016F29
:10411000000E026F000E036F10EC2EF02CC182F423
:104120000401300E8227A8EC0EF02DC182F40401A8
:10413000300E8227A8EC0EF02EC182F40401300E5E
:104140008227A8EC0EF02FC182F40401300E8227E2
:10415000A8EC0EF030C182F40401300E8227A8ECE6
:104160000EF031C182F40401300E8227A8EC0EF06B
:1041700032C182F40401300E8227A8EC0EF033C164
:1041800082F40401300E8227A8EC0EF004012C0EFC
:10419000826FA8EC0EF001013E0E006F000E016F61
:1041A000000E026F000E036F10EC2EF02CC182F493
:1041B0000401300E8227A8EC0EF02DC182F4040118
:1041C000300E8227A8EC0EF02EC182F40401300ECE
:1041D0008227A8EC0EF02FC182F40401300E822752
:1041E000A8EC0EF030C182F40401300E8227A8EC56
:1041F0000EF031C182F40401300E8227A8EC0EF0DB
:1042000032C182F40401300E8227A8EC0EF033C1D3
:1042100082F40401300E8227A8EC0EF004012C0E6B
:10422000826FA8EC0EF0200EF86EF76AF66A0401B1
:104230000900F5CF82F4A8EC0EF00900F5CF82F466
:10424000A8EC0EF00900F5CF82F4A8EC0EF00900FE
:10425000F5CF82F4A8EC0EF00900F5CF82F4A8ECBB
:104260000EF00900F5CF82F4A8EC0EF00900F5CFAE
:1042700082F4A8EC0EF00900F5CF82F4A8EC0EF061
:10428000B2EC0EF0A1EF27F08351630AD8A49FEFA0
:1042900027F08451610AD8A49FEF27F085516C0A5A
:1042A000D8A49FEF27F08651410A3FE08651440A87
:1042B0001BE08651420AD8B4A8EF21F08651350A96
:1042C000D8B42BEF29F08651360AD8B480EF29F004
:1042D0008651370AD8B4E9EF29F08651380AD8B4A4
:1042E00047EF2AF09FEF27F00798079A04017A0E0C
:1042F000826FA8EC0EF00401780E826FA8EC0EF02D
:104300000401640E826FA8EC0EF00401550E826F5A
:10431000A8EC0EF091EF21F004014C0E826FA8EC96
:104320000EF0B2EC0EF0A1EF27F00788079A040117
:104330007A0E826FA8EC0EF00401410E826FA8EC99
:104340000EF00401610E826FA8EC0EF085EF21F0F3
:104350000798078A04017A0E826FA8EC0EF0040118
:10436000420E826FA8EC0EF00401610E826FA8EC81
:104370000EF085EF21F001016667C6EF21F0676757
:10438000C6EF21F06867C6EF21F0696716D001011A
:104390004F67D2EF21F05067D2EF21F05167D2EF93
:1043A00021F052670AD00101000E006F000E016F6C
:1043B000000E026F000E036F120011B80AD0010147
:1043C000620E046F010E056F000E066F000E076F80
:1043D00009D00101A70E046F020E056F000E066FD3
:1043E000000E076F66C100F167C101F168C102F1FB
:1043F00069C103F172EC2DF003BF6FEF22F0119A47
:10440000119C0101000E046FA80E056F550E066F7A
:10441000020E076F66C100F167C101F168C102F1C8
:1044200069C103F166C18AF167C18BF168C18CF182
:1044300069C18DF172EC2DF003BF0BD00101000EAC
:104440008A6FA80E8B6F550E8C6F020E8D6F118ABE
:10445000119C0E0E3CEC0BF0E8CF18F10F0E3CEC6B
:104460000BF0E8CF19F1100E3CEC0BF0E8CF1AF18D
:10447000110E3CEC0BF0E8CF1BF1BBEC2CF08AC129
:1044800004F18BC105F18CC106F18DC107F172EC0D
:104490002DF007827FEC2CF0BBEC2CF007927FEC28
:1044A0002CF08AC100F18BC101F18CC102F18DC1E8
:1044B00003F107927FEC2CF0CC0E046FE00E056F39
:1044C000870E066F050E076F72EC2DF000C118F114
:1044D00001C119F102C11AF103C11BF140D013AAA5
:1044E00074EF22F0138E139A119C119A0101800E21
:1044F000006F1A0E016F060E026F000E036F4FC1A0
:1045000004F150C105F151C106F152C107F172EC3D
:104510002DF003AF05D06DEC2EF0118C119A120026
:104520000E0E3CEC0BF0E8CF18F10F0E3CEC0BF04C
:10453000E8CF19F1100E3CEC0BF0E8CF1AF1110E98
:104540003CEC0BF0E8CF1BF14FC100F150C101F181
:1045500051C102F152C103F107827FEC2CF018C166
:1045600000F119C101F11AC102F11BC103F11200DE
:104570000401730E826FA8EC0EF004012C0E826F02
:10458000A8EC0EF0078462C166F163C167F164C1F3
:1045900068F165C169F14BC14FF14CC150F14DC19A
:1045A00051F14EC152F157C159F158C15AF1079416
:1045B000DEEC22F0B2EC0EF0A1EF27F066C100F1C4
:1045C00067C101F168C102F169C103F1010110EC99
:1045D0002EF0D3EC2BF00401630E826FA8EC0EF0EA
:1045E00004012C0E826FA8EC0EF04FC100F150C1F7
:1045F00001F151C102F152C103F1010110EC2EF0A1
:10460000D3EC2BF00401660E826FA8EC0EF00401CF
:104610002C0E826FA8EC0EF06DEC2EF059C100F15B
:104620005AC101F1010110EC2EF0D3EC2BF0040182
:10463000740E826FA8EC0EF0120010820401530E6B
:10464000826FA8EC0EF004012C0E826FA8EC0EF025
:1046500083C32AF184C32BF185C32CF186C32DF1CA
:1046600087C32EF188C32FF189C330F18AC331F19A
:104670008BC332F18CC333F10101BBEC2EF032EC71
:104680002EF000C166F101C167F102C168F103C1FA
:1046900069F18EC32AF18FC32BF190C32CF191C322
:1046A0002DF192C32EF193C32FF194C330F195C332
:1046B00031F196C332F197C333F10101BBEC2EF017
:1046C00032EC2EF000C14FF101C150F102C151F1A5
:1046D00003C152F1AEEC2EF099C32FF19AC330F121
:1046E0009BC331F19CC332F19DC333F10101BBEC9B
:1046F0002EF032EC2EF000C159F101C15AF1DEEC7E
:1047000022F004012C0E826FA8EC0EF098EF23F03B
:10471000118E1CA002D01CAE108C1BBE02D01BA49C
:10472000108E03018251520A02E10F8201D00F92D2
:104730008251750A02E1108401D010948251550A09
:1047400002E1108601D010968351310A03E11382F1
:10475000138402D01392139411A003D011A401D09A
:104760001084078410B216EF24F010A4FAEF23F09F
:10477000BAC166F1BBC167F1BCC168F1BDC169F1E5
:10478000BEC16AF1BFC16BF1C0C16CF1C1C16DF1B5
:10479000C2C16EF1C3C16FF1C4C170F1C5C171F185
:1047A000C6C172F1C7C173F1C8C174F1C9C175F155
:1047B000CAC176F1CBC177F1CCC178F1CDC179F125
:1047C000CEC17AF1CFC17BF1D0C17CF1D1C17DF1F5
:1047D000D2C17EF1D3C17FF1D4C180F1D5C181F1C5
:1047E000D6C182F1D7C183F1D8C184F1D9C185F195
:1047F00002EF24F062C166F163C167F164C168F140
:1048000065C169F1BAC186F1BBC187F1BCC188F14C
:10481000BDC189F14BC14FF14CC150F14DC151F1B6
:104820004EC152F157C159F158C15AF107940FA026
:1048300038EF24F00101966725EF24F0976725EF04
:1048400024F0986725EF24F0996729EF24F038EFDA
:1048500024F0BBEC21F096C104F197C105F198C199
:1048600006F199C107F172EC2DF003BF65EF27F057
:10487000BBEC21F00101000E046F000E056F010E6C
:10488000066F000E076FA3EC2DF011A02AD011A225
:1048900028D010EC2EF0296701D005D004012D0E90
:1048A000826FA8EC0EF030C182F40401300E822732
:1048B000A8EC0EF031C182F40401300E8227A8EC7E
:1048C0000EF032C182F40401300E8227A8EC0EF003
:1048D00033C182F40401300E8227A8EC0EF0B2EC52
:1048E0000EF012A8C5D012981DC01EF01E3A1E422E
:1048F000070E1E1600011E50000AD8B404EF25F062
:1049000000011E50010AD8B490EF24F000011E509F
:10491000020AD8B48EEF24F036EF25F036EF25F0FA
:104920006DEC2EF02DC001F12EC000F1D8900133B6
:104930000033D890013300330101630E046F000E81
:10494000056F000E066F000E076FA3EC2DF0280E0A
:10495000046F000E056F000E066F000E076F72ECFD
:104960002DF000C130F06DEC2EF02BC001F1019F55
:10497000019D2CC000F10101A40E046F000E056F13
:10498000000E066F000E076FA3EC2DF000C12FF094
:1049900000C104F101C105F102C106F103C107F133
:1049A000640E006F000E016F000E026F000E036FA9
:1049B00072EC2DF0050E046F000E056F000E066FF1
:1049C000000E076FA3EC2DF000C104F101C105F149
:1049D00002C106F103C107F16DEC2EF030C000F109
:1049E00072EC2DF000C131F031C0E8FF050F305CF2
:1049F00003E78A8436EF25F031C0E8FF0A0F305C08
:104A000001E68A9436EF25F000C124F101C125F1B9
:104A100002C126F103C127F16DEC2EF073EC2EF0EC
:104A20001D501F0BE8CF00F10101640E046F000E52
:104A3000056F000E066F000E076F83EC2DF024C18A
:104A400004F125C105F126C106F127C107F172EC79
:104A50002DF003BF02D08A9401D08A8424C100F1D2
:104A600025C101F126C102F127C103F1A1EF27F011
:104A700000C124F101C125F102C126F103C127F1D2
:104A800010AE4DD0109E00C108F101C109F102C164
:104A90000AF103C10BF110EC2EF030C1DAF131C193
:104AA000DBF132C1DCF133C1DDF108C100F109C134
:104AB00001F10AC102F10BC103F101016C0E046F97
:104AC000070E056F000E066F000E076F72EC2DF0DB
:104AD00003BF04D00101550EDE6F1CD008C100F1E8
:104AE00009C101F10AC102F10BC103F10101A40ED8
:104AF000046F060E056F000E066F000E076F72EC56
:104B00002DF003BF04D001017F0EDE6F03D0010141
:104B1000FF0EDE6F1F8E11AE65EF27F0119E24C1D0
:104B200000F125C101F126C102F127C103F111A055
:104B300005D011A203D00FB065EF27F010A4A8EFA5
:104B400025F00401750E826FA8EC0EF0ADEF25F094
:104B50000401720E826FA8EC0EF004012C0E826F1D
:104B6000A8EC0EF010EC2EF02967BCEF25F0040144
:104B7000200E826FBFEF25F004012D0E826FA8EC8E
:104B80000EF030C182F40401300E8227A8EC0EF042
:104B900031C182F40401300E8227A8EC0EF004012A
:104BA0002E0E826FA8EC0EF032C182F40401300E9A
:104BB0008227A8EC0EF033C182F40401300E822764
:104BC000A8EC0EF004016D0E826FA8EC0EF004014B
:104BD0002C0E826FA8EC0EF04FC100F150C101F114
:104BE00051C102F152C103F1010110EC2EF0D3ECDE
:104BF0002BF00401480E826FA8EC0EF004017A0E2F
:104C0000826FA8EC0EF004012C0E826FA8EC0EF05F
:104C100066C100F167C101F168C102F169C103F128
:104C2000010110EC2EF0D3EC2BF00401630E826F27
:104C3000A8EC0EF004012C0E826FA8EC0EF066C1F9
:104C400000F167C101F168C102F169C103F101011D
:104C50000A0E046F000E056F000E066F000E076F40
:104C600083EC2DF0000E046F120E056F000E066F20
:104C7000000E076FA3EC2DF010EC2EF02AC182F489
:104C80000401300E8227A8EC0EF02BC182F404013F
:104C9000300E8227A8EC0EF02CC182F40401300EF5
:104CA0008227A8EC0EF02DC182F40401300E822779
:104CB000A8EC0EF02EC182F40401300E8227A8EC7D
:104CC0000EF02FC182F40401300E8227A8EC0EF002
:104CD00030C182F40401300E8227A8EC0EF00401EA
:104CE0002E0E826FA8EC0EF031C182F40401300E5A
:104CF0008227A8EC0EF032C182F40401300E822724
:104D0000A8EC0EF033C182F40401300E8227A8EC27
:104D10000EF00401730E826FA8EC0EF004012C0E4D
:104D2000826FA8EC0EF06DEC2EF059C100F15AC163
:104D300001F1CBEC28F013A2EDEF26F004012C0ECC
:104D4000826FA8EC0EF086C166F187C167F188C159
:104D500068F189C169F1BBEC21F00101000E046F1B
:104D6000000E056F010E066F000E076FA3EC2DF00D
:104D700010EC2EF02967C2EF26F00401200E826F9E
:104D8000C5EF26F004012D0E826FA8EC0EF030C1A5
:104D900082F40401300E8227A8EC0EF031C182F4B7
:104DA0000401300E8227A8EC0EF004012E0E826F53
:104DB000A8EC0EF032C182F40401300E8227A8EC78
:104DC0000EF033C182F40401300E8227A8EC0EF0FD
:104DD00004016D0E826FA8EC0EF013A414EF27F0FF
:104DE00004012C0E826FA8EC0EF013AC02EF27F03A
:104DF0000401500E826FA8EC0EF0139C1398139AC6
:104E000014EF27F013AE0FEF27F00401460E826F68
:104E1000A8EC0EF0139E1398139A14EF27F00401D8
:104E2000530E826FA8EC0EF038A02BEF27F0040190
:104E30002C0E826FA8EC0EF08BB026EF27F0040149
:104E4000440E826FA8EC0EF02BEF27F00401530EF6
:104E5000826FA8EC0EF00FB231EF27F00FA063EFD6
:104E600027F004012C0E826FA8EC0EF0200EF86ED5
:104E7000F76AF66A04010900F5CF82F4A8EC0EF097
:104E80000900F5CF82F4A8EC0EF00900F5CF82F40A
:104E9000A8EC0EF00900F5CF82F4A8EC0EF00900A2
:104EA000F5CF82F4A8EC0EF00900F5CF82F4A8EC5F
:104EB0000EF00900F5CF82F4A8EC0EF00900F5CF52
:104EC00082F4A8EC0EF0B2EC0EF00F90109E129847
:104ED000A1EF27F00401630E826FA8EC0EF004012D
:104EE0002C0E826FA8EC0EF0A7EC27F004012C0E1C
:104EF000826FA8EC0EF01AEC28F004012C0E826FE1
:104F0000A8EC0EF096EC28F004012C0E826FA8ECB1
:104F10000EF00101F80E006FCD0E016F660E026FEC
:104F2000030E036FBCEC27F004012C0E826FA8EC7B
:104F30000EF0ACEC28F0B2EC0EF0A1EF27F0B2ECE2
:104F40000EF00301C26B07901092B0EF2AF0D890D8
:104F50000E0E3CEC0BF0E8CF00F10F0E3CEC0BF02A
:104F6000E8CF01F1100E3CEC0BF0E8CF02F1110E8E
:104F70003CEC0BF0E8CF03F10101000E046F000ED2
:104F8000056F010E066F000E076FA3EC2DF010ECFD
:104F90002EF02AC182F40401300E8227A8EC0EF014
:104FA0002BC182F40401300E8227A8EC0EF02CC134
:104FB00082F40401300E8227A8EC0EF02DC182F499
:104FC0000401300E8227A8EC0EF02EC182F40401F9
:104FD000300E8227A8EC0EF02FC182F40401300EAF
:104FE0008227A8EC0EF030C182F40401300E822733
:104FF000A8EC0EF031C182F40401300E8227A8EC37
:105000000EF004012E0E826FA8EC0EF032C182F475
:105010000401300E8227A8EC0EF033C182F40401A3
:10502000300E8227A8EC0EF004016D0E826FA8EC02
:105030000EF01200120E3CEC0BF0E8CF00F1130E54
:105040003CEC0BF0E8CF01F1140E3CEC0BF0E8CF98
:1050500002F1150E3CEC0BF0E8CF03F101010A0E52
:10506000046F000E056F000E066F000E076F83ECD5
:105070002DF0000E046F120E056F000E066F000E6D
:10508000076FA3EC2DF010EC2EF02AC182F404017E
:10509000300E8227A8EC0EF02BC182F40401300EF2
:1050A0008227A8EC0EF02CC182F40401300E822776
:1050B000A8EC0EF02DC182F40401300E8227A8EC7A
:1050C0000EF02EC182F40401300E8227A8EC0EF0FF
:1050D0002FC182F40401300E8227A8EC0EF030C1FB
:1050E00082F40401300E8227A8EC0EF004012E0E8B
:1050F000826FA8EC0EF031C182F40401300E8227D9
:10510000A8EC0EF032C182F40401300E8227A8EC24
:105110000EF033C182F40401300E8227A8EC0EF0A9
:105120000401730E826FA8EC0EF012000A0E3CEC24
:105130000BF0E8CF00F10B0E3CEC0BF0E8CF01F1E7
:105140000C0E3CEC0BF0E8CF02F10D0E3CEC0BF03A
:10515000E8CF03F1CBEF28F0060E3CEC0BF0E8CFE4
:1051600000F1070E3CEC0BF0E8CF01F1080E3CEC2F
:105170000BF0E8CF02F1090E3CEC0BF0E8CF03F1A5
:10518000CBEF28F001016DEC2EF0078457C100F140
:1051900058C101F107940101E80E046F800E056FFC
:1051A000000E066F000E076F83EC2DF0000E046FEB
:1051B000040E056F000E066F000E076FA3EC2DF0B6
:1051C000880E046F130E056F000E066F000E076F3A
:1051D00072EC2DF00A0E046F000E056F000E066FC4
:1051E000000E076FA3EC2DF010EC2EF001012967E3
:1051F000FFEF28F00401200E826F02EF29F0040176
:105200002D0E826FA8EC0EF030C182F40401300E36
:105210008227A8EC0EF031C182F40401300E8227FF
:10522000A8EC0EF032C182F40401300E8227A8EC03
:105230000EF004012E0E826FA8EC0EF033C182F442
:105240000401300E8227A8EC0EF00401430E826F99
:10525000A8EC0EF0120087C32AF188C32BF189C392
:105260002CF18AC32DF18BC32EF18CC32FF18DC38A
:1052700030F18EC331F190C332F191C333F10101AA
:10528000296BBBEC2EF032EC2EF00101000E046F06
:10529000000E056F010E066F000E076F83EC2DF0F8
:1052A0000E0E0C6E00C10BF025EC0BF00F0E0C6E09
:1052B00001C10BF025EC0BF0100E0C6E02C10BF0CF
:1052C00025EC0BF0110E0C6E03C10BF025EC0BF06E
:1052D00004017A0E826FA8EC0EF004012C0E826F8E
:1052E000A8EC0EF00401350E826FA8EC0EF004015C
:1052F0002C0E826FA8EC0EF0A7EC27F091EF21F0B6
:1053000087C32AF188C32BF189C32CF18AC32DF1FD
:105310008BC32EF18CC32FF18DC330F18EC331F1CD
:1053200090C332F191C333F10101296BBBEC2EF034
:1053300032EC2EF0880E046F130E056F000E066F10
:10534000000E076F77EC2DF0000E046F040E056F52
:10535000000E066F000E076F83EC2DF00101E80EC2
:10536000046F800E056F000E066F000E076FA3EC32
:105370002DF00A0E0C6E00C10BF025EC0BF00B0E9D
:105380000C6E01C10BF025EC0BF00C0E0C6E02C183
:105390000BF025EC0BF00D0E0C6E03C10BF025ECA1
:1053A0000BF004017A0E826FA8EC0EF004012C0EB3
:1053B000826FA8EC0EF00401360E826FA8EC0EF09E
:1053C00004012C0E826FA8EC0EF096EC28F091EF01
:1053D00021F087C32AF188C32BF189C32CF18AC33A
:1053E0002DF18BC32EF18CC32FF18DC330F18FC300
:1053F00031F190C332F191C333F10101BBEC2EF0D6
:1054000032EC2EF0000E046F120E056F000E066FC8
:10541000000E076F83EC2DF001010A0E046F000EE1
:10542000056F000E066F000E076FA3EC2DF0120E35
:105430000C6E00C10BF025EC0BF0130E0C6E01C1CD
:105440000BF025EC0BF0140E0C6E02C10BF025ECEA
:105450000BF0150E0C6E03C10BF025EC0BF00401E4
:105460007A0E826FA8EC0EF004012C0E826FA8EC6D
:105470000EF00401370E826FA8EC0EF004012C0E22
:10548000826FA8EC0EF01AEC28F091EF21F087C3A0
:105490002AF188C32BF189C32CF18AC32DF18BC368
:1054A0002EF18CC32FF18DC330F18EC331F190C337
:1054B00032F191C333F10101296BBBEC2EF032ECD8
:1054C0002EF0880E046F130E056F000E066F000E8F
:1054D000076F77EC2DF0000E046F040E056F000EC1
:1054E000066F000E076F83EC2DF00101E80E046FCC
:1054F000800E056F000E066F000E076FA3EC2DF0F7
:10550000060E0C6E00C10BF025EC0BF0070E0C6EB6
:1055100001C10BF025EC0BF0080E0C6E02C10BF074
:1055200025EC0BF0090E0C6E03C10BF025EC0BF013
:1055300004017A0E826FA8EC0EF004012C0E826F2B
:10554000A8EC0EF00401380E826FA8EC0EF00401F6
:105550002C0E826FA8EC0EF0ACEC28F091EF21F04D
:1055600007A823EF2BF00101800E006F1A0E016FC8
:10557000060E026F000E036F4BC104F14CC105F122
:105580004DC106F14EC107F172EC2DF003BF69EF7A
:105590002BF0CDEC2BF04BC100F14CC101F14DC112
:1055A00002F14EC103F107827FEC2CF018C104F127
:1055B00019C105F11AC106F11BC107F1F80E006F00
:1055C000CD0E016F660E026F030E036F72EC2DF0AD
:1055D0000E0E0C6E00C10BF025EC0BF00F0E0C6ED6
:1055E00001C10BF025EC0BF0100E0C6E02C10BF09C
:1055F00025EC0BF0110E0C6E03C10BF025EC0BF03B
:10560000078401016DEC2EF057C100F158C101F182
:1056100007940A0E0C6E00C10BF025EC0BF00B0E7C
:105620000C6E01C10BF025EC0BF00C0E0C6E02C1E0
:105630000BF025EC0BF00D0E0C6E03C10BF025ECFE
:105640000BF069EF2BF007AA69EF2BF0078401013B
:105650006DEC2EF057C100F158C101F10794060E10
:105660000C6E00C10BF025EC0BF0070E0C6E01C1A7
:105670000BF025EC0BF0080E0C6E02C10BF025ECC4
:105680000BF0090E0C6E03C10BF025EC0BF0078438
:1056900062C100F163C101F164C102F165C103F1AE
:1056A0000794120E0C6E00C10BF025EC0BF0130EDC
:1056B0000C6E01C10BF025EC0BF0140E0C6E02C148
:1056C0000BF025EC0BF0150E0C6E03C10BF025EC66
:1056D0000BF00798079A0401805181197F0B0DE0A8
:1056E0009EA8FED714EE00F081517F0BE126E75013
:1056F000812B0F01AD6E6BEF2BF005012F51010ACD
:105700000FE081AA95EF2BF005012F51000AD8B4C4
:1057100030EF35F000011650050AD8B430EF35F0FF
:1057200081B895EF2BF09DEC2FF0E1EF0DF018C153
:1057300000F119C101F11AC102F11BC103F1000E00
:10574000046F000E056F010E066F000E076FA3ECCD
:105750002DF029A1C2EF2BF02051D8B4C2EF2BF0CD
:1057600018C100F119C101F11AC102F11BC103F105
:10577000000E046F000E056F0A0E066F000E076F15
:10578000A3EC2DF012000101045100130551011387
:10579000065102130751031312000101186B196B14
:1057A0001A6B1B6B12002AC182F40401300E82278F
:1057B000A8EC0EF02BC182F40401300E8227A8EC75
:1057C0000EF02CC182F40401300E8227A8EC0EF0FA
:1057D0002DC182F40401300E8227A8EC0EF02EC1F8
:1057E00082F40401300E8227A8EC0EF02FC182F45F
:1057F0000401300E8227A8EC0EF030C182F40401BF
:10580000300E8227A8EC0EF031C182F40401300E74
:105810008227A8EC0EF032C182F40401300E8227F8
:10582000A8EC0EF033C182F40401300E8227A8ECFC
:105830000EF012002FC182F40401300E8227A8EC72
:105840000EF030C182F40401300E8227A8EC0EF075
:1058500031C182F40401300E8227A8EC0EF032C16F
:1058600082F40401300E8227A8EC0EF033C182F4DA
:105870000401300E8227A8EC0EF01200060E216EF5
:10588000060E226E060E236E212E44EF2CF0222EE1
:1058900044EF2CF0232E44EF2CF08B84020E216E6B
:1058A000020E226E020E236E212E54EF2CF0222EB9
:1058B00054EF2CF0232E54EF2CF08B941200FF0E9B
:1058C000226E22C023F0030E216E8B84212E65EF01
:1058D0002CF0030E216E232E65EF2CF08B9422C04A
:1058E00023F0030E216E212E73EF2CF0030E216E98
:1058F000233E73EF2CF0222E61EF2CF012000101F9
:10590000005305E1015303E1025301E1002B42EC96
:105910002DF06DEC2EF03951006F3A51016F420EAF
:10592000046F4B0E056F000E066F000E076F83ECC1
:105930002DF000C104F101C105F102C106F103C15E
:1059400007F118C100F119C101F11AC102F11BC11F
:1059500003F107B2B0EF2CF077EC2DF0B2EF2CF0A2
:1059600072EC2DF000C118F101C119F102C11AF158
:1059700003C11BF112006DEC2EF059C100F15AC1A8
:1059800001F1060E3CEC0BF0E8CF04F1070E3CEC05
:105990000BF0E8CF05F1080E3CEC0BF0E8CF06F178
:1059A000090E3CEC0BF0E8CF07F172EC2DF000C1D2
:1059B00024F101C125F102C126F103C127F1290E0D
:1059C000046F000E056F000E066F000E076F83EC6C
:1059D0002DF0EE0E046F430E056F000E066F000EE5
:1059E000076F77EC2DF024C104F125C105F126C124
:1059F00006F127C107F183EC2DF000C11CF101C1B4
:105A00001DF102C11EF103C11FF1120E3CEC0BF09F
:105A1000E8CF04F1130E3CEC0BF0E8CF05F1140EC7
:105A20003CEC0BF0E8CF06F1150E3CEC0BF0E8CFA8
:105A300007F10D0E006F000E016F000E026F000ED9
:105A4000036F83EC2DF0180E046F000E056F000E2F
:105A5000066F000E076FA3EC2DF01CC104F11DC1F1
:105A600005F11EC106F11FC107F177EC2DF06A0E9A
:105A7000046F2A0E056F000E066F000E076F72ECA2
:105A80002DF01200BF0EFA6E200E3A6F396BD890CF
:105A90000037013702370337D8B053EF2DF03A2FD4
:105AA00048EF2DF039073A070353D8B412000331F9
:105AB000070B80093F6F03390F0B010F396F80EC23
:105AC0005FF0406F390580EC5FF0405D405F396BFF
:105AD0003F33D8B0392739333FA968EF2DF0405113
:105AE00039271200010192EC2EF0D8B0120001010A
:105AF00003510719346F55EC2EF0D8900751031954
:105B000034AF800F12000101346B79EC2EF0D8A075
:105B10008FEC2EF0D8B0120064EC2EF06DEC2EF06D
:105B20001F0E366FA5EC2EF00B35D8B055EC2EF0CD
:105B3000D8A00335D8B01200362F92EF2DF034B133
:105B40007CEC2EF012000101346B0451051106119A
:105B500007110008D8A079EC2EF0D8A08FEC2EF019
:105B6000D8B01200086B096B0A6B0B6BA5EC2EF01A
:105B70001F0E366FA5EC2EF007510B5DD8A4CDEFAC
:105B80002DF006510A5DD8A4CDEF2DF00551095D29
:105B9000D8A4CDEF2DF00451085DD8A0E0EF2DF092
:105BA0000451085F0551D8A0053D095F0651D8A0F2
:105BB000063D0A5F0751D8A0073D0B5FD8900081D2
:105BC000362FBAEF2DF034B17CEC2EF0346B79EC3B
:105BD0002EF0D890A9EC2EF007510B5DD8A4FDEF64
:105BE0002DF006510A5DD8A4FDEF2DF00551095D99
:105BF000D8A4FDEF2DF00451085DD8A00CEF2EF0D5
:105C0000003F0CEF2EF0013F0CEF2EF0023F0CEFA7
:105C10002EF0032BD8B4120034B17CEC2EF012001D
:105C20000101346B79EC2EF0D8B01200AEEC2EF0FE
:105C3000200E366F003701370237033711EE33F08D
:105C40000A0E376FE7360A0EE75CD8B0E76EE5520A
:105C5000372F22EF2EF0362F1AEF2EF034B1298194
:105C6000D890120001010A0E346F200E366F11EE2B
:105C700029F03451376F0A0ED890E652D8B0E72693
:105C8000E732372F3DEF2EF0033302330133003379
:105C9000362F37EF2EF0E750FF0FD8A00335D8B0DE
:105CA000120029B17CEC2EF012000451002705519E
:105CB000D8B0053D01270651D8B0063D022707514F
:105CC000D8B0073D032712000051086F0151096F3A
:105CD00002510A6F03510B6F12000101006B016B3F
:105CE000026B036B12000101046B056B066B076B03
:105CF00012000335D8A012000351800B001F011FB2
:105D0000021F031F003F8CEF2EF0013F8CEF2EF09F
:105D1000023F8CEF2EF0032B342B032512000735A6
:105D2000D8A012000751800B041F051F061F071F74
:105D3000043FA2EF2EF0053FA2EF2EF0063FA2EFA8
:105D40002EF0072B342B07251200003701370237BE
:105D50000337083709370A370B3712000101296B5F
:105D60002A6B2B6B2C6B2D6B2E6B2F6B306B316B6F
:105D7000326B336B120001012A510F0B2A6F2B512A
:105D80000F0B2B6F2C510F0B2C6F2D510F0B2D6FF9
:105D90002E510F0B2E6F2F510F0B2F6F30510F0BFA
:105DA000306F31510F0B316F32510F0B326F335156
:105DB0000F0B336F120010A806D08994000EC76E27
:105DC000220EC66E05D08984000EC76E220EC66EE6
:105DD000050EE82EFED7120010A802D0898401D04B
:105DE0008994050EE82EFED71200DBEC2EF09E966D
:105DF000C69E000EC96EFF0E9EB602D0E82EFCD7DE
:105E00009E96C69E000EC96EFF0E9EB602D0E82E6C
:105E1000FCD7C9CFAFF59E96C69E000EC96EFF0E89
:105E20009EB602D0E82EFCD7C9CFB0F59E96C69E8E
:105E3000000EC96EFF0E9EB602D0E82EFCD7C9CF69
:105E4000B1F59E96C69E000EC96EFF0E9EB602D09C
:105E5000E82EFCD7C9CFB2F59E96C69E000EC96E3D
:105E6000FF0E9EB602D0E82EFCD7C9CFB3F59E96A2
:105E7000C69E000EC96EFF0E9EB602D0E82EFCD75D
:105E8000C9CFB4F59E96C69E000EC96EFF0E9EB693
:105E900002D0E82EFCD7C9CFB5F5ECEC2EF01200FD
:105EA000DBEC2EF09E96C69E800EC96EFF0E9EB64F
:105EB00002D0E82EFCD79E96C69EAFC5C9FFFF0E46
:105EC0009EB602D0E82EFCD79E96C69EB0C5C9FFEE
:105ED000FF0E9EB602D0E82EFCD79E96C69EB1C598
:105EE000C9FFFF0E9EB602D0E82EFCD79E96C69E36
:105EF000B2C5C9FFFF0E9EB602D0E82EFCD79E9613
:105F0000C69EB3C5C9FFFF0E9EB602D0E82EFCD7D1
:105F10009E96C69EB4C5C9FFFF0E9EB602D0E82E5F
:105F2000FCD79E96C69EB5C5C9FFFF0E9EB602D091
:105F3000E82EFCD7ECEC2EF01200DBEC2EF09E9657
:105F4000C69E070EC96EFF0E9EB602D0E82EFCD785
:105F50009E96C69E000EC96EFF0E9EB602D0E82E1B
:105F6000FCD7C9CFAFF59E96C69E000EC96EFF0E38
:105F70009EB602D0E82EFCD7C9CFB0F59E96C69E3D
:105F8000000EC96EFF0E9EB602D0E82EFCD7C9CF18
:105F9000B1F59E96C69E000EC96EFF0E9EB602D04B
:105FA000E82EFCD7C9CFB2F5ECEC2EF0DBEC2EF0EE
:105FB0009E96C69E25C0C9FFFF0E9EB602D0E82E53
:105FC000FCD79E96C69E000EC96EFF0E9EB602D0EE
:105FD000E82EFCD7C9CFB6F5ECEC2EF01200DBECC6
:105FE0002EF09E96C69E870EC96EFF0E9EB602D0FC
:105FF000E82EFCD79E96C69EAFC5C9FFFF0E9EB683
:1060000002D0E82EFCD79E96C69EB0C5C9FFFF0EF3
:106010009EB602D0E82EFCD79E96C69EB1C5C9FF9B
:10602000FF0E9EB602D0E82EFCD79E96C69EB2C545
:10603000C9FFFF0E9EB602D0E82EFCD7ECEC2EF086
:10604000DBEC2EF09E96C69E26C0C9FFFF0E9EB6C4
:1060500002D0E82EFCD79E96C69EB6C5C9FFFF0E9D
:106060009EB602D0E82EFCD7ECEC2EF01200DBEC52
:106070002EF09E96C69E870EC96EFF0E9EB602D06B
:10608000E82EFCD79E96C69E000EC96EFF0E9EB6E9
:1060900002D0E82EFCD79E96C69E800EC96EFF0EDB
:1060A0009EB602D0E82EFCD79E96C69E800EC96E84
:1060B000FF0E9EB602D0E82EFCD79E96C69E800E9E
:1060C000C96EFF0E9EB602D0E82EFCD7ECEC2EF087
:1060D0001200DBEC2EF09E96C69E870EC96EFF0E58
:1060E0009EB602D0E82EFCD79E96C69E000EC96EC4
:1060F000FF0E9EB602D0E82EFCD79E96C69E000EDE
:10610000C96EFF0E9EB602D0E82EFCD79E96C69EA4
:10611000800EC96EFF0E9EB602D0E82EFCD79E966A
:10612000C69E800EC96EFF0E9EB602D0E82EFCD72A
:10613000ECEC2EF0120010A817D0DBEC2EF09E969F
:10614000C69E8F0EC96EFF0E9EB602D0E82EFCD7FB
:106150009E96C69E000EC96EFF0E9EB602D0E82E19
:10616000FCD7ECEC2EF012009DEC2FF0120010A8E2
:106170002DD0DBEC2EF09E96C69E26C0C9FFFF0EEA
:106180009EB602D0E82EFCD79E96C69E450EC96EDE
:10619000FF0E9EB602D0E82EFCD7ECEC2EF0DBEC26
:1061A0002EF09E96C69E8F0EC96EFF0E9EB602D032
:1061B000E82EFCD79E96C69E000EC96EFF0E9EB6B8
:1061C00002D0E82EFCD7ECEC2EF01200DBEC2EF027
:1061D0009E96C69E26C0C9FFFF0E9EB602D0E82E30
:1061E000FCD79E96C69E010EC96EFF0E9EB602D0CB
:1061F000E82EFCD7ECEC2EF0DBEC2EF09E96C69E43
:10620000910EC96EFF0E9EB602D0E82EFCD79E9668
:10621000C69EA50EC96EFF0E9EB602D0E82EFCD714
:10622000ECEC2EF01200DBEC2EF09E96C69E26C003
:10623000C9FFFF0E9EB602D0E82EFCD79E96C69EE2
:10624000810EC96EFF0E9EB602D0E82EFCD7ECEC94
:106250002EF01200DBEC2EF09E96C69E26C0C9FFE3
:10626000FF0E9EB602D0E82EFCD79E96C69E010E6B
:10627000C96EFF0E9EB602D0E82EFCD7ECEC2EF0D5
:106280001200DBEC2EF09E96C69E910EC96EFF0E9C
:106290009EB602D0E82EFCD79E96C69EA50EC96E6D
:1062A000FF0E9EB602D0E82EFCD7ECEC2EF01200CA
:1062B000DBEC2EF09E96C69E910EC96EFF0E9EB62A
:1062C00002D0E82EFCD79E96C69E000EC96EFF0E29
:1062D0009EB602D0E82EFCD7ECEC2EF012000501A1
:1062E000256B266B276B286B899A400EC76E200E94
:1062F000C66E9E96C69E030EC96EFF0E9EB602D057
:10630000E82EFCD79E96C69E27C5C9FFFF0E9EB6F7
:1063100002D0E82EFCD79E96C69E26C5C9FFFF0E6A
:106320009EB602D0E82EFCD79E96C69E25C5C9FF14
:10633000FF0E9EB602D0E82EFCD79E96C69EC9528E
:10634000FF0E9EB602D0E82EFCD7898A0F01C950F5
:10635000FF0A01E1120005012E51130A05E00501B3
:106360002E51170A0CE012000501F00E256FFF0EEA
:10637000266F0F0E276F000E286FC8EF31F0050152
:10638000F00E256FFF0E266FFF0E276F000E286F91
:10639000899A400EC76E200EC66E9E96C69E030E4C
:1063A000C96EFF0E9EB602D0E82EFCD79E96C69E02
:1063B00027C5C9FFFF0E9EB602D0E82EFCD79E96D9
:1063C000C69E26C5C9FFFF0E9EB602D0E82EFCD79A
:1063D0009E96C69E25C5C9FFFF0E9EB602D0E82E2A
:1063E000FCD79E96C69EC952FF0E9EB602D0E82EDE
:1063F000FCD7898A0F01C950FF0A1DE005012E5103
:10640000130A05E005012E51170A0BE012000501E1
:10641000000E256F000E266F100E276F000E286FDE
:1064200012000501000E256F000E266F000E276F6B
:10643000010E286F12000501256B266B276B286B58
:1064400005012E51130A05E005012E51170A0CE033
:1064500012000501000E216F000E226F080E236F3F
:10646000000E246F3DEF32F00501000E216F000E8B
:10647000226F800E236F000E246F21C500F122C50C
:1064800001F123C502F124C503F125C504F126C598
:1064900005F127C506F128C507F1C3EC2BF000C1B3
:1064A00025F501C126F502C127F503C128F5899A12
:1064B000400EC76E200EC66E9E96C69E030EC96E17
:1064C000FF0E9EB602D0E82EFCD79E96C69E27C52C
:1064D000C9FFFF0E9EB602D0E82EFCD79E96C69E40
:1064E00026C5C9FFFF0E9EB602D0E82EFCD79E96A9
:1064F000C69E25C5C9FFFF0E9EB602D0E82EFCD76A
:106500009E96C69EC952FF0E9EB602D0E82EFCD7BC
:10651000898AC950FF0A08E104C125F505C126F59D
:1065200006C127F507C128F5D89005012433233388
:10653000223321332151F00B216F05012167A8EF90
:1065400032F02267A8EF32F02367A8EF32F0246719
:106550003DEF32F00501100E2527E86A2623E86A90
:106560002723E86A28231200E86A05012E51130A3E
:1065700006E005012E51170A0BE0020E120005017C
:106580002851000A03E12751F00B07E0010E120029
:1065900005012851000A01E0010E120029C500F191
:1065A0002AC501F12BC502F12CC503F125C504F163
:1065B00026C505F127C506F128C507F172EC2DF0B7
:1065C00003BF1200B4EC32F0D8A446EF33F0899A3E
:1065D000400EC76E200EC66E9E96C69E060EC96EF3
:1065E000FF0E9EB602D0E82EFCD7898A899A9E9625
:1065F000C69E020EC96EFF0E9EB602D0E82EFCD7D4
:106600009E96C69E27C5C9FFFF0E9EB602D0E82EF5
:10661000FCD79E96C69E26C5C9FFFF0E9EB602D029
:10662000E82EFCD79E96C69E25C5C9FFFF0E9EB6D6
:1066300002D0E82EFCD79E96C69E000EC96EFF0EB5
:106640009EB602D0E82EFCD7898A899A9E96C69E6D
:10665000050EC96EFF0E9EB602D0E82EFCD79E96A0
:10666000C69EC952FF0E9EB602D0E82EFCD7C9B016
:106670002FEF33F0898A0501100E2527E86A2623BB
:10668000E86A2723E86A2823CEEF32F01200899ABD
:10669000400EC76E200EC66E9E96C69E060EC96E32
:1066A000FF0E9EB602D0E82EFCD7898A899A9E9664
:1066B000C69EC70EC96EFF0E9EB602D0E82EFCD74E
:1066C000898A0501256B266B276B286B1200899A36
:1066D000400EC76E200EC66E9E96C69E050EC96EF3
:1066E000FF0E9EB602D0E82EFCD79E96C69EC952DB
:1066F000FF0E9EB602D0E82EFCD7C9CF37F5898AA7
:106700001200899A400EC76E200EC66E9E96C69ED7
:10671000B90EC96EFF0E9EB602D0E82EFCD7898A4C
:106720001200899A400EC76E200EC66E9E96C69EB7
:10673000AB0EC96EFF0E9EB602D0E82EFCD7898A3A
:10674000FF0EE82EFED71200B4EC32F0D8A41200EF
:10675000899A400EC76E200EC66E9E96C69E030E88
:10676000C96EFF0E9EB602D0E82EFCD79E96C69E3E
:1067700027C5C9FFFF0E9EB602D0E82EFCD79E9615
:10678000C69E26C5C9FFFF0E9EB602D0E82EFCD7D6
:106790009E96C69E25C5C9FFFF0E9EB602D0E82E66
:1067A000FCD79E96C69EC952FF0E9EB602D0E82E1A
:1067B000FCD7898A0F01C950FF0AD8A4A3EF34F08F
:1067C0000501FE0E376F37A037998BA0379BF5EC8C
:1067D0002EF0AFC538F5B0C539F5B1C53AF5B2C53B
:1067E0003BF5B3C53CF5B4C53DF5B5C53EF50784ED
:1067F000BAC166F1BBC167F1BCC168F1BDC169F145
:106800004BC14FF14CC150F14DC151F14EC152F14C
:1068100057C159F158C15AF1BBEC21F000C13FF505
:1068200001C140F502C141F503C142F505016167AF
:1068300021EF34F0626721EF34F0636721EF34F029
:10684000646725EF34F032EF34F061C504F162C5BE
:1068500005F163C506F164C507F172EC2DF003BFC5
:10686000A3EF34F059C143F55AC144F5B9C545F514
:10687000BAC546F507940501110E326F899A400E8C
:10688000C76E200EC66E9E96C69E060EC96EFF0E81
:106890009EB602D0E82EFCD7898A899A9E96C69E1B
:1068A000020EC96EFF0E9EB602D0E82EFCD79E9651
:1068B000C69E27C5C9FFFF0E9EB602D0E82EFCD7A4
:1068C0009E96C69E26C5C9FFFF0E9EB602D0E82E34
:1068D000FCD79E96C69E25C5C9FFFF0E9EB602D068
:1068E000E82EFCD725EE37F0322F02D083EF34F0BC
:1068F0009E96C69EDECFC9FFFF0E9EB602D0E82E42
:10690000FCD774EF34F0898A899A9E96C69E050E4C
:10691000C96EFF0E9EB602D0E82EFCD79E96C69E8C
:10692000C952FF0E9EB602D0E82EFCD7C9B08EEF3A
:1069300034F0898A0501100E2527E86A2623E86AC3
:106940002723E86A2823120021C500F122C501F19E
:1069500023C502F124C503F1899A400EC76E200EAB
:10696000C66E9E96C69E0B0EC96EFF0E9EB602D0D8
:10697000E82EFCD79E96C69E02C1C9FFFF0E9EB6AA
:1069800002D0E82EFCD79E96C69E01C1C9FFFF0E1D
:106990009EB602D0E82EFCD79E96C69E00C1C9FFC7
:1069A000FF0E9EB602D0E82EFCD79E96C69EC95218
:1069B000FF0E9EB602D0E82EFCD725EE37F005017B
:1069C000100E326F9E96C69EC952FF0E9EB602D022
:1069D000E82EFCD7C9CFDEFF322FE2EF34F0898AF0
:1069E0001200899A400EC76E200EC66E9E96C69EF5
:1069F000900EC96EFF0E9EB602D0E82EFCD79E9672
:106A0000C69E000EC96EFF0E9EB602D0E82EFCD7C1
:106A10009E96C69E000EC96EFF0E9EB602D0E82E50
:106A2000FCD79E96C69E000EC96EFF0E9EB602D083
:106A3000E82EFCD79E96C69EC952FF0E9EB602D087
:106A4000E82EFCD7C9CF2DF59E96C69EC952FF0EE3
:106A50009EB602D0E82EFCD7C9CF2EF5898A120047
:106A60008B903EEC2CF0B9C5E8FFD70802E33EEC72
:106A70002CF0B9C5E8FFC80802E33EEC2CF0B9C51C
:106A8000E8FFB90802E33EEC2CF0B9C5E8FFAA081C
:106A900002E33EEC2CF0B9C5E8FF9B0802E33EECB4
:106AA0002CF081EC33F0F29CF29E8B94C69AC2904B
:106AB0009482948C720ED36ED3A4FED789968A905A
:106AC0009390F29AF2949D909E909D929E92F2984D
:106AD000F2929BEC30F0FF0EE8CF00F0E82EFED7EC
:106AE000002EFCD7F290F286815081A87AEF35F023
:106AF000F29E0300700ED36EF296F290010E376E86
:0A6B000003805FEC2CF071EF0BF046
:10BF0000E844F926000C160C2B0C3F0C520C640C68
:10BF1000760C860C960CA50CB30CC10CCF0CDC0C6B
:06BF2000E80CF40C000C1B
:0200000400F00A
:0100C800FE39
:00000001FF
